:102000000030002099280000C52500007124000040
:10201000712400007124000071240000712400006C
:10202000712400007124000071240000712400005C
:10203000712400007124000071240000C92D0000EB
:10204000712400007124000071240000712400003C
:10205000712400007124000071240000712400002C
:102060004930000071240000712400007124000038
:10207000712400007124000071240000712400000C
:1020800071240000712400007124000071240000FC
:1020900071240000712400007124000071240000EC
:1020A00071240000712400007124000071240000DC
:1020B00071240000712400007124000071240000CC
:10240000FFFFFFFFFFFFFFFFFFFFFFFFFFE4FEFFF8
:1024100010B5064C2378002B07D1054B002B02D0BA
:10242000044800E000BF0123237010BD10F0FF1F1F
:102430000000000088AA000008B5084B002B03D05C
:102440000748084900E000BF07480368002B03D095
:10245000064B002B00D0984708BDC0460000000086
:1024600088AA000014F0FF1F10F0FF1F00000000FA
:10247000FFBE7047FFBE7047FFBE7047FFBE70478C
:10248000FFBE7047FFBE7047FFBE7047FFBE70477C
:10249000FFBE7047FFBE7047FFBE7047FFBE70476C
:1024A000FFBE7047FFBE7047FFBE7047FFBE70475C
:1024B000FFBE7047FFBE7047FFBE7047FFBE70474C
:1024C000FFBE7047FFBE7047FFBE7047FFBE70473C
:1024D000FFBE7047FFBE7047FFBE7047FFBE70472C
:1024E000FFBE7047FFBE7047FFBE7047FFBE70471C
:1024F000FFBE7047FFBE7047FFBE7047FFBE70470C
:10250000FFBE7047FFBE7047FFBE7047FFBE7047FB
:10251000FFBE7047FFBE7047FFBE7047FFBE7047EB
:10252000FFBE7047FFBE7047FFBE704720280DDC1E
:10253000C317DB0EC0181F221040C31A0120984099
:10254000C022034B5200985018607047C046FCE709
:1025500000E100E020280BDCC317DB0EC0181F22AF
:102560001040C31A034901209840802288507047C8
:10257000C046FCE700E100E030B5032915DC202867
:1025800013DCC417A40F2018FF2382101A40074D34
:1025900092005219032528408901041B1940234049
:1025A000DB00994013681943116030BD00E400E07E
:1025B000034AD2231B01D15889008908D1507047A2
:1025C00000E000E008B500F0A9F908BD08B50B4B24
:1025D0008022596992010A435A61596802220A43CA
:1025E0005A60596804220A435A60596808220A430B
:1025F0005A60FFF7DDFF62B608BDC04600800440A8
:102600000D4A3F2113788B43402B0FD0802B08D0ED
:10261000002B01D00020704713785A07FAD403200A
:10262000F9E75078C006C00F0430F4E75078C006D0
:10263000C00F0130EFE7C04600400640F0B55F46EE
:1026400056464D464446F0B45C4F05017C5B83B072
:10265000FFF7D6FF7D195A4980230F220235234008
:1026600022400F26AA468B460193304043001B1898
:102670005B009B185B00FB18188A904200D17FE03A
:10268000311C4E4C01408B00E3189B6D5D781C782B
:10269000A8469D781B79A9469C46052937D889000C
:1026A0005D466B589F46474B454647495D706546BA
:1026B0000D701C70019B002B04D00C1C0121237891
:1026C0001942FCD03F4D10242B793E491C42FBD1CE
:1026D000CD7801234C469C432B402343CB700528E7
:1026E00017D99042C1D103B03CBC90469946A2464E
:1026F000AB46F0BD334B10211C701C1C23791942D2
:10270000FCD0304B45465D702F4B61461970052853
:10271000E7D801238340092119423BD130211942D6
:1027200041D106211942DCD0264C0C2123790B40E3
:10273000042BFBD1904298D1D5E7224D2C70102468
:102740002B7920491C42FBD043464B70CD780123A6
:102750004C469C432B402343CB701B4B64461C7060
:10276000D5E7184B65461C7044465C70164C2570C6
:1027700001990029CBD0012123781942FCD0C6E76A
:10278000534699785D781C781B798946A8469C4603
:10279000011C82E70B4C0C2123791942FCD1904299
:1027A00000D062E79FE7074C0C2123790B40082BF0
:1027B000FBD1904200D058E795E7C046E89E000064
:1027C000D09E0000004006400050064038B50A493F
:1027D0000A4B0B4A0B4CD1500B4B03229A8080259D
:1027E00001225A706D0420221A7000206562FFF7E2
:1027F00025FF656238BDC04600200000080D0000BE
:1028000000E000E000800440002005407047C04622
:1028100030B588421AD0002A18D00324012506E0DA
:10282000032A08D908C9043A08C0002A0ED00B1C94
:1028300003431C42F4D01D4209D1012A07D90B8859
:10284000023A038002310230002AF0D130BD0B7809
:10285000013A037001310130E7E7C04638B50A4C50
:102860000025002C06D138BD9A68002AFBD0FFF75E
:10287000CFFF0C35631919685868002901D1002869
:10288000F2D09A68F3E7C046B0AA00007047C0468D
:102890007047C0467047C04638B5FFF7F7FFFFF7EF
:1028A00095FF184B181C002805D0854681B00020E4
:1028B000C043009001B0144B144AD21A08D1FFF75C
:1028C000CDFFFFF7E7FF0020114907F00DF9FEE704
:1028D000032501240020291C194006D1032A04D90C
:1028E00002C3043A002AF6D1E9E7211C194005D1B8
:1028F000012A03D91980023A0233F3E71870013A2A
:102900000133EFE70030002010F0FF1F54F8FF1FE5
:102910002CF0FF1F08B5FFF7BFFFC0467047C04649
:10292000094B022201215A7008209A600022197076
:1029300098705960DA601A611A755A759A75DA7565
:102940001A765A769A767047F4F0FF1F10B5C823AE
:10295000114C1B0223606360104B1148A36001F00F
:1029600019FCE0600F4801F015FC012222761621C7
:10297000E27780226176120203210023A17622628F
:102980000821C82220616361E37623776177A3770A
:102990006262A36210BDC046B8F0FF1FF380000062
:1029A00050C300008813000010B51F4B9B7E012B05
:1029B00004D81E4B01219A698A439A611B4B8021DE
:1029C0009A6901208A439A619969194A0A409A6171
:1029D0009969184A0A409A61174A9169814391613D
:1029E00091690220814391615A6980200005024368
:1029F0005A615A69802189050A435A615C698022BB
:102A0000D20514435C615C682043586098680143B8
:102A1000996059680A435A60084B8022596812032A
:102A20000A435A6010BDC046F4F0FF1F00F00F408B
:102A3000FFFFFEFFFFFFFDFF40F00F40008004405E
:102A4000074B8022596992050A435A61054B0922B6
:102A50009A6000225A605A6840218A435A6070473F
:102A60000080044000B00340014B00221A807047F0
:102A700014F1FF1F30B5144B9B7E012B1FD9134B54
:102A80000122DA600B221A6002250122104B0F4945
:102A90009B5C1F221340402213430B6080220B6873
:102AA0001A42FCD00B4C0948002301695A00090561
:102AB000090D0133A152DAB2AA42F6D330BD034B5D
:102AC0000022DA600125E1E7F4F0FF1F00B00340C7
:102AD000A09F000010F1FF1F08B5174B9A7E012A36
:102AE00024D9164A01219069014391619B7E0222FB
:102AF00093430FD000F020FD00F02EFD0F4B8022FD
:102B0000996952020A439A619969802292020A43A2
:102B10009A6108BD00F018FD084B094A99690A40FE
:102B20009A619969074A0A409A61F2E7034A0120CB
:102B3000916981439161D9E7F4F0FF1F00F00F40E4
:102B4000FFFFFEFFFFFFFDFF024B802292059A6010
:102B50007047C04600F00F40024B802292055A6039
:102B60007047C04600F00F40024B80229205DA60A9
:102B70007047C04600F00F40024B8022D2059A6099
:102B80007047C04600F00F40024B8022D2055A60C9
:102B90007047C04600F00F40024B8022D205DA6039
:102BA0007047C04600F00F407047C0467047C046AF
:102BB00000207047024B01201B6918407047C04637
:102BC00000F00F40024B802212055A607047C04649
:102BD00000F00F40024B802212059A607047C046F9
:102BE00000F00F40024B18690001C00F7047C0464B
:102BF00000F00F40052821D8114B80001B589F463C
:102C0000104B01201B69184070470E4B1869800754
:102C1000C00FF9E70C4B01201B691840F4E70A4B81
:102C20001869C003C00FEFE7074B18698003C00F96
:102C3000EAE7054B18690006C00FE5E70020E3E767
:102C4000889F000040F00F4000F00F4000207047C8
:102C50007047C0467047C046002807D0012801D001
:102C600000207047034B588880B2FAE7014B188860
:102C700080B2F6E710F1FF1F002806D0012801D02E
:102C800000207047024B5888FBE7014B1888F8E793
:102C900014F1FF1F002804D0012801D1024B5980F4
:102CA0007047014B1980FBE714F1FF1F1D4B0821F2
:102CB0005A6870B58A435A601B4B10225969002626
:102CC0000A435A619969194A00250A4080219A618C
:102CD00010200A22490398601C690C4201D001357A
:102CE000EDB258601C690C4201D10136F6B2013ACE
:102CF000D2B2002AEFD10A2D0ED00D4B00221A704D
:102D0000094B8022996952030A439A61054B0822B4
:102D100059680A435A6070BD0A2EEED1044B012255
:102D20001A70EDE70080044000F00F40FFFFEFFF56
:102D3000B5F0FF1F30B5124B83B01B78002B01D1CB
:102D400003B030BDFFF7ECFDFFF700FE0D480E4964
:102D500000F0BEFB80250D498024AD05E4050C4A3A
:102D60008D6000208C60CD60CC600190019B93420F
:102D7000F9D8019B01330193019B9342F9D9F2E702
:102D8000B5F0FF1FF4F0FF1FB8F0FF1F00F00F4079
:102D90001FA10700044B054900221A6059609A6080
:102DA00007221A607047C04610E000E0204E000085
:102DB000014B00221A60704710E000E0014B1868D8
:102DC0007047C04658F0FF1F044B1A6801321A6062
:102DD000034B1A6801321A607047C04658F0FF1F53
:102DE000F8F3FF1F08B5FFF7F1FB08BD304B70B5D6
:102DF0005D69802424022C432E4E5C6134780123CB
:102E000023433370012573782A4C1D42FBD063782D
:102E100003252B4080252B4363701C23E370082877
:102E200003D8254B80001B589F46224B8320987067
:102E3000204BCC0849010020C9B2E4B2D8721C74FE
:102E4000597407219874D874187559759875D87580
:102E5000002A0BD0D4085201E4B2D2B21C765A76C2
:102E60009876D876187759779877D87711490122CC
:102E70000B7893430B704B781A42FCD170BD0D4B0D
:102E800081209870D4E70B4BB1209870D0E7094BA4
:102E900093209870CCE7074B89209870C8E7054BC2
:102EA00087209870C4E7034B80209870C0E7C04625
:102EB0000080044000400240A49F0000F0B54F464F
:102EC0004646C0B4284B041C1879012210403AD061
:102ED0002121585C0825284039D062702020185CD8
:102EE0005E5C595C400589462221595C84468846CF
:102EF00040466546C001284323215F5C8046802010
:102F00000506404628437F087609B6043843304317
:102F10004D4607263540ED03284360605B5C1A4050
:102F2000A2700023114910485A181179E218013390
:102F30001172082BF6D12C23C35C0F22134023708F
:102F40000123037101200CBC90469946F0BD6070CE
:102F500020229A5C585CD2004009024362605B5CAC
:102F6000DB06DB0FA370DCE700400240204002409C
:102F7000F0B5334B041C98790122104031D09A727D
:102F8000616800292EDBC908C9B2302299546568EE
:102F90003122995C6801172529400143C9B299542F
:102FA000995C0820814399540023E218254E117A38
:102FB0009A19013322481171082BF6D13C23C25CC7
:102FC0000F218A4321780A43C2546368002B30DB07
:102FD0003123C25C10218A43C254194B01229A71D9
:102FE0000120F0BDC900090E302019546668312156
:102FF000585C750018270740EE0C0820074376013F
:1030000037436D036E0F3D1C3543EDB25D5465686B
:103010006E04360E32255E5533255F5D66683A4094
:1030200076003243D2B25A555A5C1043C0B258545B
:10303000BAE73323C25C01218A43C254CDE7C046BC
:10304000004002403040024010B53F4A0223D17890
:103050000B43D3703D4B1978C9B2022921D0032903
:1030600014D0012900D010BD5C78987884423ED2FB
:10307000D078014254D159785868C9B24C1CE4B296
:103080005C7041180B78DBB21371ECE7917810207B
:10309000814391701279D968D2B20A7002221A70F3
:1030A000E1E7187C597C88421AD2587C197C411A75
:1030B000012941D0597C1A7C8A1A022A04DC224A4E
:1030C00008219078014391701A7CD968D2B2501CC3
:1030D000C0B218741C4B8A181B79DBB21370C2E79C
:1030E000917820208143917000221A70BBE7597AB1
:1030F0009078C9B2002908D12024A043907090781C
:103100001024A04390701970ADE704210143917021
:10311000997AC9B2117100225A7203221A70A2E779
:1031200090782024A043907090781024A043907051
:10313000002219721A7096E79178202081439170CD
:1031400000221A70B6E7C046006006405CF0FF1F20
:103150000D4A802351695B020B4310B553610B4B41
:1031600000215020997098710220D870D0682024D6
:10317000A043D06003225A70C0229A70082059716F
:10318000FFF7D4F910BDC04600800440006006403F
:1031900030B5104C0023D2B223726372A2706370F8
:1031A00001220D4B6160227099780825A94399701E
:1031B0009D781021294399709D78202129439043BF
:1031C000997018712378002BFCD1207A4342584122
:1031D000C0B230BD5CF0FF1F0060064010B5114C5E
:1031E0000023D2B2237263726274237403232370A8
:1031F0000D4BE1609A7808218A439A7099781022E1
:103200000A439A70997820220A439A700122104347
:1032100018712378002BFCD1207A43425841C0B268
:1032200010BDC0465CF0FF1F0060064070B5144C36
:1032300000260125D2B226726572A270049AE3605C
:10324000D3B266706374012303432674A3720D4BDB
:10325000616025709A7808218A439A7099781022C3
:103260000A439A70997820220A43A8439A701871E9
:103270002378002BFCD1207A43425841C0B270BD64
:103280005CF0FF1F006006400D4B8022596912035D
:103290000A435A610B4B1C22197882B00A431A70F8
:1032A00011229A7059796A46C9B2D17107321278DF
:1032B00000225A70197840220A431A7002B07047EF
:1032C0000080044000700740F8B50F1C161C002455
:1032D000002801D0201CF8BDFFF77CFC094D2024FC
:1032E000EB7808481C42FBD04771C3785BB2002BD7
:1032F000FBDA044B5C79E4B2002EEBD0FFF762FC02
:10330000E8E7C0460070074010B5FFF757FD041C02
:10331000FFF754FD031BDA179B185340062BF7DD0C
:1033200010BDC04610B582B001AC030A6070211C0C
:103330000222A0202370FFF72BFF211C0222A020D5
:10334000FFF74CFF207802B010BDC04600B583B037
:1033500001AB020A1A70587099700322191CA02040
:10336000FFF716FFFFF7D0FF03B000BD30B583B005
:103370000D1C141C01A9020A0A7048700222A02028
:10338000FFF706FF291C221CA020FFF727FF03B030
:1033900030BDC046F0B5574645464E46E0B4884677
:1033A0008AB0171E25D00F21013A0023002401AD59
:1033B0008946924605E0A2450CD00134BC4218D0A3
:1033C000131C4646315DEA1891705A1C861849460E
:1033D0003142F0D1020A2A706870DA1C291CA02040
:1033E0000134FFF7D5FEFFF78FFFB0B20022BC42D9
:1033F000E6D10AB01CBC90469946A246F0BDC04634
:1034000008B5C300181A80231B01C01880B2072218
:10341000FFF7C0FF08BDC04608B5C300181A8023D7
:103420001B01C01880B20722FFF7A0FF08BDC046ED
:1034300010B5C3008022181A120182B080180C1C2B
:1034400080B207226946FFF791FF6B461A7823780E
:1034500000209A4201D002B010BD6B465A786378C2
:103460009A42F8D16B469A78A3789A42F3D16A4689
:10347000D378019AE17812021A43237960791B020A
:1034800000040B430343A07900060343D01A4342D0
:103490005841E0E770B58AB001AD69462B1C263172
:1034A00000221A7001338B42FBD180248026240134
:1034B000B601230A6C70291C2222A02020342B7014
:1034C000FFF766FEFFF720FFB442F2D10AB070BDED
:1034D00038B5051C16480C1CFFF724FF642822D0C1
:1034E000FFF74AFB12480021FFF730FFFFF7D2FF3A
:1034F0000020291C1C22FFF74DFF4020211C2C22FC
:10350000FFF748FF0A486421FFF720FFFFF73CFB65
:10351000291C00201C22FFF729FF4020211C2C22FF
:10352000FFF724FF38BD034B1B78002BD8D1EFE702
:10353000FF070000B5F0FF1F08B5802200203A21E8
:10354000520200F0F9F808BD08B500203A21002227
:1035500000F0F2F808BDC046F0B5474680B4504CC4
:1035600082B0226A0020002A02D0656A002D13D1A1
:10357000382100F0F1F84B4B021C1A400020382192
:1035800000F0DAF8802200203A21520200F0D4F84C
:1035900002B004BC9046F0BD00F0D2FA236A98460F
:1035A0000823181A8540281C06F0F0F94246D31764
:1035B000041CD01858400D1C06F0E8F9021C0B1C26
:1035C000201C291C04F08AFF304B2F4A061C0F1CBC
:1035D00005F0EEFB6A46041C0D1C06F0CBFA2C4AE3
:1035E0002C4B04F0AFFA00281AD0201C291C06F03E
:1035F00099F94246041C002A10DB0020382100F013
:10360000ABF8284B021C1A400020382100F094F837
:1036100000203A21221C00F08FF8B9E74442ECE781
:10362000301C391C6A4606F0A5FA4346041C0D1CE2
:1036300000980199002B14DD06F074F9164A174B17
:103640000604291C201C05F0B3FB06F06BF9041CD2
:1036500034430020382100F07FF88022D20002435A
:10366000D2E706F05FF90C4A0C4BC643291C201C1C
:1036700005F09EFB06F056F90B4C3604241A344331
:10368000E7E7C046C046C046000000000000F0402A
:103690000000000000000000000000000088C3409F
:1036A000B8F0FF1FFFFBFFFF1027000008B5002048
:1036B000392100F051F808BD08B5021C392100205D
:1036C00000F03AF808BDC046F8B54F464646C0B4CB
:1036D00098460E1C08AB8021041C91461F7831438C
:1036E00009AB00221D78FFF7EFFD4946201C0022A0
:1036F000FFF7EAFD4146201C0022FFF7E5FD391CDB
:10370000201C0022FFF7E0FD291C201C0122FFF7EE
:10371000DBFD4A461302424613431B021F437F232D
:103720003F021E40034B3D43B600F5500CBC904693
:103730009946F8BD1CF1FF1F30B5151283B0140E69
:103740001314EDB2D2B20192DBB20095221CFFF746
:10375000BBFF03B030BDC04670B5284B7F250D4080
:103760005B5D0522041C1A4203D1254BAD00E858CD
:1037700070BD291C0022FFF7A7FD00210022201C9C
:10378000FFF7A2FD00210022201CFFF79DFD002174
:103790000022201CFFF798FD00210122201CFFF7CA
:1037A00093FD291C0022201CFFF78EFD0021002222
:1037B000201CFFF789FD002106020022201CFFF7D4
:1037C00083FD002106430022201CFFF77DFD360209
:1037D00006430021201C0122FFF776FD3602331C30
:1037E0000343222D02D0181C422DC1D1181C030204
:1037F000BED5FF231B061843BAE7C046C89F00008A
:103800001CF1FF1F10B5FFF7D9FA041CFFF7D6FA19
:10381000031BDA179B185340C72BF7DD3E4C0020E3
:10382000E27E637E12041B021A43A37E10211A4318
:10383000FFF782FFA268394BA07F1340227F01214E
:103840000A400140090752040A43A3601343627F00
:103850000820801A0F22104000061A1C02436C2117
:103860000020FFF769FF002070212D4AFFF764FF59
:10387000002020210022FFF75FFF00202D210022E1
:10388000FFF75AFF002021210022FFF755FF0020FB
:1038900023210122FFF750FF00202421214AFFF7B6
:1038A0004BFF214A00202521FFF746FF606806F004
:1038B0006DF8164B144A04F011FE06F033F8262179
:1038C000021C0020FFF738FF206806F05FF8104A5E
:1038D000104B04F003FE06F025F82721021C0020FF
:1038E000FFF72AFF00202821104AFFF725FF0020BC
:1038F0002A210C4AFFF720FF00202B211022FFF77E
:103900001BFF10BDC046C0467CE68F1EC4BC4640AF
:103910004C030000D012E33FB8F0FF1FFFFFFDE0B3
:10392000C800050032020000C5A7000065040000C1
:1039300070B51A4B00241C70194E1A4B82B01C70C3
:103940003378051C002B20D1174A01231370002D5A
:1039500010DB002201930092002020210023FFF7BA
:10396000B3FEEB17EA185A4000202721FFF7E4FEC8
:1039700002B070BD00230093022301930020202198
:1039800000220023FFF7A0FEEBE7084B00201A6897
:103990002621FFF7D1FE3470D6E7C046B4F0FF1FF2
:1039A00020F3FF1FE4F0FF1F18F1FF1F1CF3FF1FA0
:1039B000094A08B500231370084A00201370084B09
:1039C00001221A7027210022FFF7B6FE00202021D5
:1039D0000122FFF7B1FE08BDB4F0FF1FE4F0FF1FA6
:1039E00018F1FF1F10B50D4B01241C700C4B82B059
:1039F0000020272100221C70FFF79EFE00202621B8
:103A0000084AFFF799FE002300930194002020212B
:103A10000022FFF759FE02B010BDC04618F1FF1F8B
:103A200020F3FF1FFFFF000070B5154C82B0237814
:103A3000051C0E1C002B19D1124C2378002B06D02C
:103A400000202721321CFFF777FE002323702A1C59
:103A500000202D21FFF770FE00230093019300202A
:103A600020210022FFF730FE02B070BD064B00207F
:103A70001A682621FFF760FE00232370DCE7C046AA
:103A800020F3FF1F18F1FF1F1CF3FF1FF0B5154CAB
:103A900083B02378051C0F1C161C002B19D1124C67
:103AA0002378002B06D0002027213A1CFFF744FE84
:103AB00000232370721900202D21FFF73DFE002303
:103AC00000930193002020210022FFF7FDFD03B0A9
:103AD000F0BD064B00201A682621FFF72DFE0023BB
:103AE0002370DCE720F3FF1F18F1FF1F1CF3FF1FFB
:103AF00038B50D1C0021041CFFF72EFE054B021CDF
:103B00001A4001231D40AD002A43201C0021FFF76D
:103B100013FE38BDFBFF030038B50D1C6C21041CDF
:103B2000FFF71AFE054B021C1A400F231D402D06FD
:103B30002A43201C6C21FFF7FFFD38BDFFFFFFF07B
:103B400008B56C21FFF708FE0001000F08BDC04654
:103B500038B50D1C6C21041CFFF7FEFD054B021C43
:103B60001A4001231D402D072A43201C6C21FFF71A
:103B7000E3FD38BDFFFFFFEF08B56C21FFF7ECFD5B
:103B8000C000C00F08BDC04638B50D1C6C21041C18
:103B9000FFF7E2FD002D06D1054A0240201C6C21F2
:103BA000FFF7CAFD38BD802292020243F6E7C04605
:103BB000FFFFFDFF08B56C21FFF7CEFD8003C00FAE
:103BC00008BDC04638B50D1C6C21041CFFF7C4FDB0
:103BD0000F23021C9A432B401A43201C6C21FFF731
:103BE000ABFD38BD38B50D1C6C21041CFFF7B4FDCE
:103BF0007023021C9A4307231D402D012A43201CD9
:103C00006C21FFF799FD38BD38B50D1C6C21041CE3
:103C1000FFF7A2FD054B021C1A400F231D40ED01CA
:103C20002A43201C6C21FFF787FD38BD7FF8FFFF7A
:103C300038B50D1C6C21041CFFF78EFD054B021CD2
:103C40001A4003231D40ED032A43201C6C21FFF77B
:103C500073FD38BDFF7FFEFF38B50D1C6C21041CC1
:103C6000FFF77AFD054B021C1A400F231D402D055E
:103C70002A43201C6C21FFF75FFD38BDFFFF0FFFBB
:103C800038B50D1C6C21041CFFF766FD002D06D114
:103C9000054A0240201C6C21FFF74EFD38BD8022F2
:103CA000D2050243F6E7C046FFFFFFBF38B50D1C43
:103CB0006C21041CFFF750FD002D06D1054A02407F
:103CC000201C6C21FFF738FD38BD8022120302430F
:103CD000F6E7C046FFFFF7FF38B50D1C6C21041C4A
:103CE000FFF73AFD002D06D1054A0240201C6C2149
:103CF000FFF722FD38BD8022D2020243F6E7C0461C
:103D0000FFFFFBFF38B50D1C6C21041CFFF724FDE1
:103D1000002D06D1054A0240201C6C21FFF70CFD46
:103D200038BD8022D2010243F6E7C046FFBFFFFF45
:103D300038B50D1C6C21041CFFF70EFD002D06D1BB
:103D4000054A0240201C6C21FFF7F6FC38BD80229A
:103D500092010243F6E7C046FFDFFFFF38B50D1CB6
:103D60006C21041CFFF7F8FC002D06D1054A024027
:103D7000201C6C21FFF7E0FC38BD80225201024379
:103D8000F6E7C046FFEFFFFF38B50D1C6C21041CA1
:103D9000FFF7E2FC2B070AD4084A024007231D4024
:103DA0002D012A43201C6C21FFF7C6FC38BD70236F
:103DB0008022984312010243F0E7C0468FF7FFFFCD
:103DC00038B50D1C6C21041CFFF7C6FC054B021C0A
:103DD0001A400F231D40ED012A43201C6C21FFF7E0
:103DE000ABFC38BD7FF8FFFF08B56C21FFF7B4FCD2
:103DF0000F23184008BDC04608B56C21FFF7ACFC86
:103E00004006400F08BDC04608B56C21FFF7A4FC72
:103E10004005000F08BDC04608B56C21FFF79CFCAB
:103E2000C003800F08BDC04608B56C21FFF794FCA5
:103E30000002000F08BDC04608B56C21FFF78CFCDE
:103E40004000C00F08BDC04608B56C21FFF784FCD8
:103E50000003C00F08BDC04608B56C21FFF77CFC0D
:103E60004003C00F08BDC04608B56C21FFF774FCC5
:103E70004004C00F08BDC04608B56C21FFF76CFCBC
:103E80008004C00F08BDC04608B56C21FFF764FC74
:103E9000C004C00F08BDC04608B56C21FFF75CFC2C
:103EA000031C4006400F1A0501D50823184308BD1E
:103EB00008B56C21FFF750FC4005000F08BDC04657
:103EC00038B50D1C6D21041CFFF746FC6023021C55
:103ED0009A4303231D406D012A43201C6D21FFF7E7
:103EE0002BFC38BD38B50D1C6D21041CFFF734FCCC
:103EF000054B021C1A4003231D406D032A43201C5E
:103F00006D21FFF719FC38BDFF9FFFFF38B50D1C71
:103F10006D21041CFFF720FC054B021C1A400F23E7
:103F20001D402D022A43201C6D21FFF705FC38BDE2
:103F3000FFF0FFFF38B50D1C6D21041CFFF70CFCD2
:103F40000F23021C9A432B401A43201C6D21FFF7BC
:103F5000F3FB38BD38B50D1C6D21041CFFF7FCFBCD
:103F6000044B021C1A402D042A43201C6D21FFF72C
:103F7000E3FB38BDFFFF00FF38B50D1C6D21041CAD
:103F8000FFF7EAFB002D06D1054A0240201C6D21F7
:103F9000FFF7D2FB38BD802212020243F6E7C0468B
:103FA000FF7FFFFF38B50D1C6D21041CFFF7D4FB0C
:103FB000002D06D1054A0240201C6D21FFF7BCFBF5
:103FC00038BD802252040243F6E7C046FFFFFFFEE1
:103FD00008B56D21FFF7C0FB4006800F08BDC04645
:103FE00008B56D21FFF7B8FB4004800F08BDC0463F
:103FF00008B56D21FFF7B0FB0005000F08BDC046F6
:1040000008B56D21FFF7A8FB0F23184008BDC04677
:1040100008B56D21FFF7A0FB0314FF2018401A0616
:1040200001D5014B184308BD00FFFFFF08B56D2106
:10403000FFF792FB0004C00F08BDC04608B56D2114
:10404000FFF78AFBC001C00F08BDC04638B50D1C84
:104050007021041CFFF780FB054B021C1A40032350
:104060001D402D052A43201C7021FFF765FB38BD3C
:10407000FFFFCFFF38B50D1C7021041CFFF76CFB50
:10408000002D06D1054A0240201C7021FFF754FB89
:1040900038BD802212030243F6E7C046FFFFF7FF58
:1040A00038B50D1C7021041CFFF756FB002D06D1FE
:1040B000054A0240201C7021FFF73EFB38BD8022DC
:1040C000D2020243F6E7C046FFFFFBFF38B50D1CE6
:1040D0007021041CFFF740FB054B021C1A40032310
:1040E0001D402D042A43201C7021FFF725FB38BDFD
:1040F000FFFFFCFF38B50D1C7021041CFFF72CFBE3
:10410000044B021C1A402D022A43201C7021FFF789
:1041100013FB38BDFF00FFFF38B50D1C7021041CD8
:10412000FFF71AFBFF23021C9A432A43201C70212D
:10413000FFF702FB38BDC04608B57021FFF70CFB46
:104140008002800F08BDC04608B57021FFF704FB50
:104150000003C00F08BDC04608B57021FFF7FCFA88
:104160004003C00F08BDC04608B57021FFF7F4FA40
:104170008003800F08BDC04608B57021FFF7ECFA38
:10418000000AC0B208BDC04608B57021FFF7E4FAC6
:10419000C0B208BD08B500280ADB05F0F7FB0B4BE1
:1041A000094A04F09BF905F0DBFD05F0BBFB08BDF7
:1041B00005F0ECFB054B044A04F090F905F01CFDFA
:1041C00005F0B0FBF3E7C0464C030000D012E33F1C
:1041D00008B505F0DBFB054B034A04F07FF905F059
:1041E000BFFD05F09FFB08BD7CE68F1EC4BC4640AA
:1041F00008B500280ADB05F0C9FB0C4B0A4A04F09D
:10420000D7FD05F0F9FC05F08DFB08BD05F0BEFB00
:10421000064B054A04F0CCFD05F0A2FD05F082FB3B
:10422000F3E7C046C046C0464C030000D012E33F4F
:1042300008B503F0DBFD05F0E7FB064B044A04F08C
:10424000B7FD05F0D9FC05F06DFB08BDC046C046C2
:104250007CE68F1EC4BC46407047C046C046C04680
:10426000F0B54D465F4656464446F0B4002083B054
:104270003521FFF771FAC34A051C137E590641D553
:10428000012146080E4001408846D16812693F244A
:1042900052421C405BB24F429146002B40DBFEF77E
:1042A00089FC431E9841C0B28346002C23D0042CC5
:1042B0003DD9082C1FD8B44A137892460F2B1AD830
:1042C000B24A9B00D3589F465B46002B13D1073C54
:1042D000012C09D951464A6803239A4301231A4302
:1042E00000203421FFF728FA4A465042FFF720FB0E
:1042F0000A2351460B7003B03CBC90469946A24637
:10430000AB46F0BD01210E1C064040080140884626
:104310003F2411691C405BB2D7688946002BBEDA86
:10432000FEF748FC43425841C0B28346BDE7964A77
:1043300013789246111C0F2BDDD8954A9B00D35859
:104340009F46534634215A680020FFF7F5F90023B1
:1043500051460B70CFE78F4B0122002034211A7099
:10436000FFF7FAF952465060062C00D1E9E0082C1C
:1043700000D1E6E0042352461370BCE7062C00D1BE
:10438000C6E1082C00D1AFE1381CFFF7D1FA0323B6
:1043900052461370AFE7631F012B00D88BE15B46D9
:1043A000002BA8D00C2351460B70A4E7052C00D19C
:1043B000A3E1072C00D18EE17842FFF7B9FA05237B
:1043C0005246137097E75A46002A94D021210020C4
:1043D000FFF7C2F95346986051460B230B708AE7EA
:1043E0005A46002A00D086E721210020FFF7B4F9C1
:1043F00051464A6803239A43041C34210020FFF7E6
:104400009BF9002027214A46FFF796F95246926809
:104410002D21A018C20F121852100020FFF78CF99E
:104420005B46009301932021002300200022FFF728
:104430004BF90D2351460B705DE7631F012B00D82C
:1044400043E15A46002A00D155E7072351460B7035
:1044500051E75A46002A00D04DE7073C012C09D904
:1044600051464A6803239A4302231A430020342109
:10447000FFF762F94846FFF75BFA0A2352461370CA
:1044800039E7AA0500D436E70E2351460B70002009
:104490002121FFF761F9404B18600020FFF748FA2F
:1044A00000202D210022FFF747F9002021210022C2
:1044B000FFF742F9002039210022FFF73DF91AE702
:1044C0004246002A00D116E721210020FFF744F9D7
:1044D000324B5146186004230B700CE74B680122E5
:1044E0001A4334210020FFF727F97842FFF720FA1A
:1044F000052351460B70FEE6002E00D1FBE6FFF7C8
:1045000071FA062352461370F5E651464A680323B2
:104510009A4300203421FFF70FF94846FFF708FAC5
:10452000072352461370E6E600203421FFF714F902
:104530005246184B5060023C01221A70012C00D9DF
:1045400018E7022351460B70D5E64B6802221A4346
:1045500034210020FFF7F0F8381CFFF7E9F90323B6
:1045600051460B70C7E6002E00D0C4E60020FFF7CE
:10457000DFF94B465842FFF7DBF9082351460B7031
:10458000B9E6C046B8F0FF1F70F0FF1F48A000005A
:1045900088A0000018F1FF1FE8F0FF1FB0F0FF1F18
:1045A000002E00D1A7E621210020FFF7D5F8041C3A
:1045B0000020FFF7BDF9624B002019680A1B514625
:1045C0001A604A6803239A433421FFF7B5F80020A4
:1045D00027214A46FFF7B0F800202D21221CFFF7C3
:1045E000ABF8002300930193002200202021FFF765
:1045F0006BF80923524613707DE6AB0500D47AE6CA
:1046000021210020FFF7A8F84E4B033C1860002042
:10461000FFF78EF900202D210022FFF78DF80020F2
:1046200021210022FFF788F8002039210022FFF71E
:1046300083F8012C77D90E2351460B705BE6002ED0
:1046400000D158E60B230B7055E6002E00D052E641
:1046500021210020FFF780F8041C0020FFF768F9F3
:1046600051464A6803239A4300203421FFF764F837
:10467000002027214A46FFF75FF8E20F1219521077
:1046800000202D21FFF758F8002200230096019604
:1046900000202021FFF718F80D23524613702AE658
:1046A000AB0500D427E6C6E70020FFF741F90E234B
:1046B000524613701FE64346002B00D16FE6062CCE
:1046C00039D00F235246137015E6002E00D1B8E6FC
:1046D000052CF6D135E751464A6803239A4300205A
:1046E0003421FFF729F867E651464A6803239A43C5
:1046F00000203421FFF720F846E651464A6803239C
:104700009A4301231A4300203421FFF715F853E69A
:1047100051464A6803239A4302231A430020342156
:10472000FFF70AF830E649464842FFF701F90A2345
:1047300052461370DFE5042351460B70DBE5C0469B
:10474000B0F0FF1FE8F0FF1F034B1A78002A01D1D9
:1047500001221A707047C04670F0FF1F034B1A7891
:10476000002A01D00F221A707047C04670F0FF1F58
:10477000014B18787047C04670F0FF1F08B5074A14
:10478000074B11780520D9701168DA79090A1206E9
:104790000A435A6000F0A4FE08BDC04690F3FF1F14
:1047A00030F3FF1F0A4B9A78002A08D15B78142B4C
:1047B00009D8084A9B001168074A995002E0074B44
:1047C00004221A707047054B03221A70FAE7C0469C
:1047D00030F3FF1F90F3FF1F3CF3FF1F0CF4FF1F8C
:1047E00008B5074A074B11780920D9701168DA79A2
:1047F000090A12060A435A6002F064FA08BDC0466C
:1048000090F3FF1F30F3FF1F064B01221A70064B77
:104810005A78012A05D15A68D9781202034B0A4303
:104820001A607047FCF3FF1F30F3FF1FC4F3FF1F34
:10483000014B02221A707047FCF3FF1F074A002346
:104840001370074A1360074A1360074A1370074A38
:104850001360074A1360074A13607047FCF3FF1F99
:10486000C4F3FF1F04F4FF1F2CF3FF1F90F3FF1F7F
:104870001CF4FF1F38F3FF1F014B00221A70704712
:10488000FCF3FF1F30B52A4A5378012B25D0002BAB
:1048900015D0022B05D0032B0DD1264B0A225A60CE
:1048A00030BD254B00221A60244B191C283104C34B
:1048B0008B42FCD1F4E71F4B03221A70F0E71E492C
:1048C0000B68092B2DD8581C08605168D078090254
:1048D0001A4A9B0001439950E2E7174D29680029C5
:1048E000DED016485468D378026824021C430023A3
:1048F000A2421AD001338B42D2D09A008258A242EF
:10490000F8D14C1E9C420AD901339B008900C31880
:10491000401819681A1F043311608342F9D12C60C2
:10492000BEE7044B09221A70BAE70023E9E7C04644
:1049300030F3FF1F0CF4FF1F00F4FF1FC8F3FF1F2D
:1049400010B5364B5A78092A65D8354992008A58ED
:104950009746344B1A68D1431960334B082200291B
:1049600055D019689143196010BD5968DA78090269
:104970002C4B11431960F0E75968DA78294B09028A
:1049800011431A6889181960E7E75968254AD878E9
:10499000090213680143591A1160DEE75968DA7891
:1049A000204B090211431A6851431960D5E7596831
:1049B0001C4CDA7809021143206803F051F820609A
:1049C000011CCAE75968174CDA78090220681143BC
:1049D00003F09CF82160C0E75968124AD8780902B0
:1049E0001368014319401160B7E759680D4AD87838
:1049F00009021368014319431160AEE75968094A77
:104A0000D87809021368014359401160A5E7196875
:104A10000A431A60A8E7034B19689EE730F3FF1FAB
:104A2000C8A0000090F3FF1F38F3FF1F10B5324BF2
:104A30005B780A2B55D8314A9B00D3589F46304BA0
:104A40001968304B1960304B082200294FD0196883
:104A50009143196010BD2A4A2A4B106819681860E2
:104A60001160F0E7264B274A11681A68511819603F
:104A7000E9E7234B234A11681A68511A1960E2E7E3
:104A80001F4B204A11681A6851431960DBE71C4C20
:104A90001C4B2068196802F0E3FF2060011CD2E77C
:104AA000174C184B2068196803F030F82160CAE7EA
:104AB000134B144A11681A6811401960C3E7104B70
:104AC000104A11681A6811431960BCE70C4B0D4A73
:104AD00011681A6851401960B5E70A4B1968CA4352
:104AE0001A60074B08221968074B0029AFD11968D3
:104AF0000A431A60AEE7C04630F3FF1FF0A0000083
:104B000090F3FF1F1CF4FF1F38F3FF1F154B5B785A
:104B1000052B08D8144A9B00D3589F46134B144AC0
:104B200019680A401A607047104B80221968914337
:104B30001960F8E70D4B0F2219680A401A60F2E776
:104B40000A4B1022196891431960ECE7074B2022A9
:104B5000196891431960E6E7044B402219689143B4
:104B60001960E0E730F3FF1F1CA1000038F3FF1FBE
:104B7000FFFEFFFF164BDA785B681B021343154AF2
:104B8000126893420CDA144B0321186888430421FD
:104B900001431960002A0ED0082291431960704722
:104BA00093420CD00C4B0521186888430221014325
:104BB0001960002AF0D1082211431960EFE7064B73
:104BC000062118688843012101431960E2E7C046C5
:104BD00030F3FF1F90F3FF1F38F3FF1F83070DD43F
:104BE0000A4BDA785B681B021343094A934209DCDB
:104BF000084A04211170084A136002E0074B08229A
:104C00001A707047054B04221A70FAE730F3FF1F41
:104C1000FE070000FCF3FF1F28F3FF1F0CF4FF1F2B
:104C2000014B00221A707047FCF3FF1F08B50A4BB6
:104C30005A78002A09D19A78002A06D15A68D97878
:104C4000064B12020A439A4200D008BD044B0122CF
:104C50001A70FEF76FF8F8E730F3FF1FD204000078
:104C6000B5F0FF1F164B5B78012B1CD0002B0DD02D
:104C7000022B06D0032B03D1124B1A68124B5A6039
:104C80007047124B1A68104B5A60F9E7104A0E4BE6
:104C90001278DA710F4A12789A710F4A1268110A63
:104CA00059711A71ECE70A4A074B1278DA71094A0E
:104CB00012789A71094A1268110A59711A71DFE75C
:104CC00030F3FF1F1CF4FF1F0CF4FF1F90F3FF1FB6
:104CD000FCF3FF1F2CF3FF1F28F3FF1FC4F3FF1F7C
:104CE000014B02221A70704794F3FF1F034B5A685E
:104CF000D9781202024B0A431A60704730F3FF1F43
:104D0000C4F3FF1F274B5A780C2A0DD8264992006E
:104D10008A589746254A1268D10505D55A68D97828
:104D20001202234B0A431A607047204A1268110688
:104D3000F4D4F9E71D4A12681107EFD5F4E71B4ACE
:104D40001268D107EAD4EFE7184A12681107EBD5C9
:104D5000E4E7164A1268D107E0D5E5E7134A12687E
:104D60005107DBD4E0E7114A116805221142D5D181
:104D7000DAE70E4A12689107D0D4D5E70B4A1268D9
:104D80009107CBD1D0E7094A1268D106C6D4CBE748
:104D9000064A12689106C1D4C6E7044A1268510651
:104DA000BCD4C1E730F3FF1F34A1000038F3FF1F6C
:104DB000C4F3FF1F084A1368072B0CD8591C116055
:104DC000064A074910689B005850064BD9785B6823
:104DD0001B020B431360704704F4FF1FC4F3FF1F53
:104DE000A4F3FF1F30F3FF1F70B51D4B01221D4CB4
:104DF0001A701D4B20705868DE781C4B000282B080
:104E00003043984202DC151C0D400AD0184B00229A
:104E1000D91D1A7001338B42FBD12378237202B063
:104E200070BD694680B2FEF7F7FA69460A7862708B
:104E30004B78A3708B78E3708B7923714B79637116
:104E40000B79A371CB78211CE3710831A31C01E01D
:104E50001A780133AD18EDB225728B42F8D1DEE736
:104E600094F3FF1F98F3FF1F30F3FF1FFF070000AD
:104E700099F3FF1F054B1A68002A06D0013A1A6001
:104E8000034B9200D258034B1A60704704F4FF1F83
:104E9000A4F3FF1FC4F3FF1F30B5144C83B0657833
:104EA000002D0FD0012D04D0114B03221A7003B036
:104EB00030BDA3782A2BF7D1E11C0E480422FEF75F
:104EC00069FAF4E704220B4801A9FEF74FFA636878
:104ED000E2781B021343019A934202D0044B5D60B7
:104EE000E5E7034B01225A60E1E7C04630F3FF1FBC
:104EF0000CF4FF1FFB070000014B00221A707047E3
:104F0000FCF3FF1F70B5134C134D2378134E6B70D9
:104F10006168E3780A0213436B603068104B984273
:104F200005D907232B700F4B00221A7070BD80B279
:104F3000211CFEF765FA3088211CFEF779FA00285B
:104F400005D033680133336065232B70EEE7072308
:104F50002B70EBE730F3FF1F0CF4FF1F28F3FF1F4C
:104F6000FF070000FCF3FF1F70B5364E364D337857
:104F7000002B10D16968EB780A0213435A1C5ED0EB
:104F80009A00D318314A5B001360FDF717FF304BCE
:104F90001860012333706C78012C24D0002C40D091
:104FA000022C11D0032C0ED1A8783521FEF7D4FBAA
:104FB000022404400FD1254D2A68002A1FD1254B19
:104FC0001A68013A1A6070BDA8783521FEF7C4FB53
:104FD00001240440EFD0002333701F4B10221968C6
:104FE00091431960EFE7A8783521FEF7B5FB8024DF
:104FF000A4000440EFD1154D2A68002ADFD0FDF748
:10500000DDFE134B1B68C01AC317C01858402B682D
:105010009842D4D9104B1022196834700A431A6090
:10502000D1E7FDF7CBFE0A4B1B68C01AC317C018A7
:105030005840064B1B689842C1D93470C3E7074BF0
:105040001B689DE72CF3FF1F30F3FF1F24F8FF1FA1
:10505000F0F3FF1FC4F3FF1F38F3FF1F90F3FF1F90
:105060000B4B9A78002A0AD15A78142A0BD859681F
:10507000D8780902074B92000143D15002E0064B59
:1050800004221A707047044B03221A70FAE7C046D4
:1050900030F3FF1F3CF3FF1F0CF4FF1F154B9A78F2
:1050A000002A0CD15A78144B142A1AD813499200AA
:1050B00052585A60124A1278002A07D170470E4B94
:1050C00004221A700E4A1278002AF7D05B680D4A43
:1050D0001360002B08D00C4B08221968914319600B
:1050E000ECE703221A70EDE7074B082219680A4320
:1050F0001A60E3E730F3FF1F0CF4FF1F3CF3FF1FC0
:10510000F5F3FF1F90F3FF1F38F3FF1F10B50B4B94
:105110009A78002A06D15C78142C07D9084B032210
:105120001A7002E0064B04221A7010BD00202121E3
:10513000FEF712FB034BA400E050F6E730F3FF1F2D
:105140000CF4FF1F3CF3FF1F08B5044B1878FDF764
:1051500083FD034B5843000B08BDC04654F0FF1FAE
:1051600026020000014B18687047C0464CF8FF1F2C
:10517000014B18687047C04644F8FF1F014B186880
:105180007047C04640F8FF1F014B18687047C04683
:1051900038F8FF1F014B18687047C04648F8FF1FDA
:1051A000014B18687047C0462CF8FF1F014B186868
:1051B0007047C04634F8FF1F014B18687047C0465F
:1051C00030F8FF1F014B18687047C0463CF8FF1FBE
:1051D000014B18687047C04628F8FF1F014B186044
:1051E0007047C0464CF8FF1F014B18607047C0461F
:1051F00044F8FF1F014B18607047C04640F8FF1F7E
:10520000014B18607047C04638F8FF1F014B18600B
:105210007047C04648F8FF1F014B18607047C046F2
:105220002CF8FF1F014B18607047C04634F8FF1F71
:10523000014B18607047C04630F8FF1F014B1860E3
:105240007047C0463CF8FF1F014B18607047C046CE
:1052500028F8FF1F00000000014B18687047C04687
:105260007CF0FF1FF8B5FDF7A9FD514C6368C01A2B
:10527000C317C01858400A2821DC00203521FEF74A
:105280006BFA061C430641D44A4D6B69002B48D18A
:10529000237B002B60D1AB6A002B01D0730569D54D
:1052A00000200121FEF758FAC30705D4FDF76CFC76
:1052B0000020FEF7D5FFF8BDFDF75EFCF8E7FDF72F
:1052C0007DFD2121061C0020FEF746FAA368051C7F
:1052D000C01A02F08BFD6368071CF01A02F086FD0D
:1052E000011C381C02F05CFC04F08EFB2F4B2E4A94
:1052F00003F05EFD04F016FB35212060002066609F
:10530000A560FEF729FA061C4306BDD5FDF734FC5F
:10531000FEF768FB284B274D01221A706B69002BA2
:10532000B6D000202221FEF717FAC317C018584044
:105330006B699842ACD9237B002BACD1342100207F
:10534000FEF70AFA8022D200024334210020FEF741
:10535000F3F9012323739EE734210020FEF7FCF9C3
:10536000164B021C1A4000203421FEF7E5F90023F9
:10537000237390E739210020FEF7EEF92121041C68
:105380000020FEF7E9F9241AE317E4185C40AB6A41
:105390009C4200D884E7FEF725FB094B01221A70D6
:1053A0007EE7C046C046C0462D431CEBE2369A401D
:1053B0007CF0FF1FB8F0FF1FE4F0FF1FFFFBFFFFB3
:1053C000B4F0FF1FC046C046314AF8B50023137041
:1053D000304A1370304A1360304A1360304A136009
:1053E000304A1360304A1370304B8022D200991833
:1053F0001D1C002204C38B42FCD12D4E337E002B9A
:105400000DD02C4F00240437D9239B00E018391904
:1054100080B204220434FDF7A9FF502CF4D1737E2E
:10542000002B0BD10024A0229200A018291980B2D1
:1054300004220434FDF79AFFE02CF4D1B37D002B55
:105440001CD01D4B01221A701C4C2068FEF7A2FED6
:105450001B4B18606068FEF7BBFE1A4B01221860F8
:10546000194B1A70E27F002A0BD0184A5A60184A6A
:105470009A60184ADA60184A1A61F8BD0E4A137029
:10548000E2E7164A5A609A60DA601A61F5E7C046A8
:1054900050F8FF1FF4F3FF1FC4F3FF1F90F3FF1F2B
:1054A0001CF4FF1F38F3FF1F2CF3FF1F20F4FF1F16
:1054B000F4F0FF1F3CF3FF1FFCF3FF1FB8F0FF1FCA
:1054C00024F3FF1F1CF3FF1F8CF0FF1F954100000A
:1054D000F1410000D141000031420000594200007A
:1054E00030B5CD4C83B0A378002B04D16378CB4A80
:1054F0009B00D3589F46CA4C0423237006280DD125
:10550000C84B1B78002B09D06368C74A1360002B77
:1055100006D0C64B082219689143196003B030BD0C
:10552000C24B0822186802431A60F7E7052801D128
:1055300000F06EFF062801D101F028FA072801D0FB
:105540000828EBD1B64B03221A70E7E7052801D1F2
:1055500000F0E4FD0628F1D1B54BB14CDB7F636070
:10556000CEE7052801D100F03DFE062801D100F06C
:10557000E5FE072801D101F018FB0828CED11A203A
:10558000FDF7D0FEAB4B9876A54B5860C6E70528D3
:1055900001D100F001FE062801D100F0DBFE072852
:1055A00001D101F02CFB0828B8D1A34C04226020C3
:1055B000211CFDF7DBFE2268994B5A60AEE70528F7
:1055C000C0D00628BAD100206F21FEF7C5F8944C50
:1055D000000E606094E70528B4D00628AED1904C48
:1055E00000236360954B1A78002A01D00122626083
:1055F00000221A70924B1A78002A03D060680222A7
:105600000243626000221A707AE7052801D100F097
:1056100013FF062892D111210020FEF79DF804F017
:10562000B5F97C4B7A4A03F0C3FB04F0E5FA7C4CF5
:1056300004F078F9606063E7052801D100F097FD78
:10564000062801D100F0A0FE072801D101F0B7FA29
:10565000082800D062E77B4C04226820211CFDF75B
:1056600085FE22686E4B5A6058E7052801D100F08C
:1056700076FF062800D061E7FEF718F8684C6060F6
:105680003EE7052800D15DE7062800D056E7002058
:105690006F21FEF761F8624C83059B0D63602FE775
:1056A000052801D100F0FEFE062801D101F060F9C5
:1056B000072801D101F0C5F9082800D02EE7624C77
:1056C0004C20211C0422FDF751FE604B20689B6892
:1056D0009847534B586021E7052801D100F057FD4A
:1056E000062801D100F030FE072801D101F07DFA33
:1056F000082800D012E75820FDF714FE4C4B18760E
:10570000474B58600AE7052801D100F052FD0628F2
:1057100000D013E70020FEF71FFD414C6060EFE66C
:10572000052801D100F09DFE062800D006E70020E4
:105730003821FEF711F83A4C6060E1E6052801D106
:1057400000F073FD062800D0F8E60020FEF70CFDFF
:10575000334C6060D4E6052800D1F3E6062800D07B
:10576000ECE60020011CFDF7F7FF042318402C4C49
:1057700000D15FE701236360C2E6052801D100F094
:1057800048FD062800D0D9E60020FEF7DDFC244CB9
:105790006060B5E6052801D100F017FD062801D1AB
:1057A00000F0F8FD072801D101F0BCF9082800D06D
:1057B000B4E6274C04226420211CFDF7D7FD2268A3
:1057C000174B5A60AAE6052801D100F05FFE0628B3
:1057D00000D0B3E60020FEF7AFFC114C60608FE60E
:1057E000052801D100F058FE062800D0A6E60020CA
:1057F000FEF7CAFC0A4C606082E6052800D1A1E6EB
:10580000062800D09AE6134B054C1B68636077E6C8
:1058100073989E1FB5F8044030F3FF1F68A1000085
:105820000CF4FF1FF5F3FF1F90F3FF1F38F3FF1F6A
:10583000B8F0FF1FF4F0FF1FD8F0FF1FE4F0FF1FC8
:10584000B4F0FF1FE0F0FF1FC4F0FF1F8CF0FF1F3C
:10585000DCF0FF1FB0F0FF1F052800D172E606281C
:1058600000D06BE600207121FDF776FFD14C60601F
:1058700046E6052801D100F05AFE062800D05DE674
:105880000020FEF779FCCB4C606039E6052800D19A
:1058900058E6062800D051E6C74BC64C1B6863602B
:1058A0002EE6052801D100F011FE062801D101F0F5
:1058B00075F8072801D101F08EF8082800D02DE6F0
:1058C000BE4C5020211C0422FDF750FDBC4B20682B
:1058D0009B689847B74B586020E6052801D100F037
:1058E000D2FC062800D029E613210020FDF734FF62
:1058F000B04C011E28D0B34802F064F86060B24B8F
:10590000DB7F002B00D0FBE56068FEF743FC6060A6
:10591000F6E5052801D100F073FF062800D00DE65A
:105920000020FEF7A9FAA34C6060E9E5052801D143
:1059300000F0C4FC062800D000E614210020FDF78A
:105940000BFF9C4C011ED6D1A04B6360D7E7052806
:1059500001D100F0E8FC062800D0EFE5984B954C0B
:105960001B786360CCE5052800D1EBE5062800D064
:10597000E4E5FFF7E9FB8F4C6060C1E5052801D144
:1059800000F0ACFE062800D0D8E50020FEF76CFA47
:10599000002801D001F067F9A078FEF72DFA854CB8
:1059A0006060ADE5052801D100F084FE062800D036
:1059B000C4E50020FEF758FA002801D001F05AF99A
:1059C000A078FEF721FA7B4C606099E5052801D1AB
:1059D00000F0A7FD062800D0B0E50020FEF754FA3D
:1059E000744C60608CE5052801D100F0DCFD0628D0
:1059F00000D0A3E50020FEF737FA6E4C60607FE52B
:105A0000052801D100F0B3FD062800D096E56C4BC7
:105A1000252100209C68FDF79FFEA047654C606033
:105A20006EE5052801D100F058FF062800D085E575
:105A30000020FEF7EDFA5F4C606061E5052801D1BA
:105A400000F0C2FE062800D078E500203421FDF7E2
:105A500083FE584C0307DB0F636051E5052801D135
:105A600000F0C3FD062800D058E5FFF79FFB514C1E
:105A7000606045E5052800D164E5062800D05DE5B5
:105A800000203521FDF768FE4A4C8305DB0F63607B
:105A900036E5052800D159E3062800D04EE54A4BEB
:105AA0005869474B9B689847424C606028E5052839
:105AB00000D147E5062800D040E500206F21FDF722
:105AC0004BFE3C4CC302DB0E636019E5052801D197
:105AD00000F0F6FC062800D030E50020FEF7BCF907
:105AE000344C60600CE5052801D100F017FE062853
:105AF00000D023E50020FEF7A7F92E4C6060FFE4FC
:105B0000052801D100F0F0FC062800D016E50020A1
:105B10003421FDF721FE274C0305DB0F6360EFE422
:105B2000052801D100F04DFD062800D006E5002033
:105B3000FEF772F91F4C6060E2E4052801D100F025
:105B4000D9FD062800D0F9E400203421FDF704FE39
:105B50000223184C03405A4253416360D0E40528A5
:105B600001D100F09EFE062800D0E7E40020FEF7F9
:105B70003FFA104C6060C3E4052801D100F0D4FD69
:105B8000062800D0DAE40E4B2B2100209C68FDF79C
:105B9000E3FDA047074C6060B2E4052801D100F0A6
:105BA0000FFC062800D0B9E4FFF7E8FA014C60606A
:105BB000A6E4C0460CF4FF1FE8F0FF1FC8F0FF1F6B
:105BC0008CF0FF1F80969800B8F0FF1FFFFFFF00CA
:105BD000052801D100F01AFE062801D100F0C4FE0C
:105BE000072801D100F019FF082800D096E4EA4BFD
:105BF000DA7F002A01D101F044F81A68E74B5A60B5
:105C00008CE4052801D100F07AFE062800D095E446
:105C10000020FEF709F9E14C606071E4052801D12C
:105C200000F022FD062801D100F094FE072801D1E2
:105C300000F034FF082800D070E4D74BDA7ED74B51
:105C40005A606BE4052801D100F063FC062800D0FF
:105C500064E4FFF7B7FAD14C606051E4052800D145
:105C60009EE3062800D059E4FFF7B2FACB4C6060FF
:105C700046E4052801D100F0E7FD062800D05DE4E8
:105C800000203421FDF768FDC44CC306DB0F6360C0
:105C900036E4052801D100F02CFE062800D04DE4A2
:105CA0000020FEF7ADF9BD4C606029E4052800D165
:105CB0001FE3062800D041E415210020FDF74CFD2C
:105CC000B64C011E00D13FE615E6052801D100F0D3
:105CD0009CFC062800D021E4FFF75CFAAF4C606022
:105CE000FFF70EFC052800D180E3062801D100F063
:105CF00043FE072801D100F05EFE082801D0FFF71F
:105D00000DFCA54B5A7EA54B5A60FFF707FC0528F2
:105D100001D100F000FE062801D100F002FE0728A4
:105D200001D100F0CBFE082801D0FFF7F7FB9A4B1A
:105D30001A7F9A4B5A60FFF7F1FB052801D100F05A
:105D4000A5FC062801D0FFF7F9FB00203421FDF760
:105D500003FD924C4307DB0F6360FFF7D1FB05287F
:105D600001D100F0B3FC062801D0FFF7D7FBFFF705
:105D700023FA8A4C6060FFF7C3FB052801D1FFF7C7
:105D8000E1FB062801D0FFF7D9FB00203521FDF704
:105D9000E3FC824C8307DB0F6360FFF7B1FB052850
:105DA00001D100F00BFD062801D0FFF7C7FB002052
:105DB000FEF73CF9794C6060FFF7A2FB052801D1A2
:105DC00000F069FD062801D0FFF7B8FB0020FEF7C0
:105DD0000BF8724C6060FFF793FB052801D100F0CF
:105DE0006CFD062801D0FFF7A9FB0020FEF7F8F8AC
:105DF0006A4C6060FFF784FB052801D100F0C2FC0B
:105E0000062801D0FFF79AFB654B2A2100201C6968
:105E1000FDF7A2FCA047614C6060FFF771FB05280D
:105E200000D1C5E2062801D0FFF778FBFFF79AF909
:105E30005A4C6060FFF764FB052800D101E2062898
:105E400001D0FFF77BFB564B272100209C68FDF714
:105E500083FCA047514C6060FFF752FB052801D13D
:105E600000F053FD062801D0FFF768FB0020FDF786
:105E7000E3FF4A4C6060FFF743FB052801D1FFF7C1
:105E800061FB062801D0FFF759FBFFF7E5F9434C0A
:105E90006060FFF735FB052801D100F0A9FC06285A
:105EA00001D0FFF73BFBFFF77BF93C4C6060FFF74D
:105EB00027FB052800D17CE3062801D0FFF72EFB45
:105EC000FFF762F9354C6060FFF71AFB052800D137
:105ED0005BE3062801D0FFF731FB314B2421002082
:105EE0001C69FDF739FCA0472C4C6060FFF708FBEC
:105EF000052801D100F0F7FC062801D0FFF71EFBB2
:105F00000020FEF79BF8254C6060FFF7F9FA0528A2
:105F100001D100F017FC062801D0FFF70FFB204B42
:105F2000332100209C68FDF717FCA0471B4C6060E4
:105F3000FFF7E6FA052800D15FE3062801D0FFF756
:105F4000EDFAFFF715F9154C6060FFF7D9FA05284F
:105F500001D100F08DFC062801D100F0E9FC0728F2
:105F600001D100F08AFD082801D0FFF7D7FA0A4BCB
:105F70009A7E0A4B5A60FFF7D1FA052801D100F04A
:105F800096FC062801D0FFF7D9FA0020FEF720F88A
:105F9000024C6060FFF7B4FAB8F0FF1F0CF4FF1F6B
:105FA0008CF0FF1F052801D100F0FAFB062801D074
:105FB000FFF7C4FAEA4B232100209C68FDF7CCFBD5
:105FC000A047E84C6060FFF79BFA052800D1FEE28D
:105FD000062801D100F0B5FC072801D100F07CFDB6
:105FE000082801D0FFF79AFADF4B5A7FDD4B5A6041
:105FF000FFF794FA052801D1FFF7A4FA062801D08B
:10600000FFF79CFA00203521FDF7A6FBD54C0123B4
:1060100018406060FFF774FA052801D1FFF792FA83
:10602000062801D0FFF78AFAFCF7C4FDCD4C60606A
:10603000FFF766FA052801D100F045FC062801D0DB
:10604000FFF77CFA00201121FDF786FBC54C60604C
:10605000FFF756FA052800D1BAE1062801D0FFF76C
:106060006DFABF4B282100201C69FDF775FBA04786
:10607000BC4C6060FFF744FA052801D1FFF762FAD3
:10608000062801D0FFF75AFAB54B222100209C6860
:10609000FDF762FBA047B34C6060FFF731FA0528BB
:1060A00000D1BAE2062801D0FFF748FA00203421D7
:1060B000FDF752FBAB4C012383436360FFF720FAEB
:1060C000052800D1BDE2062801D100F06BFC0728AD
:1060D00001D100F08EFC082801D0FFF71FFAA24B77
:1060E000DA7F002A01D100F0B7FD5A689D4B5A6053
:1060F000FFF714FA052800D194E1062801D0FFF734
:106100001DFA00202121FDF727FB964C6060FFF768
:10611000F7F9944C03232370FFF7F0F96368E278F2
:106120001B02134301D100F0F3FC012B01D000F05E
:10613000EAFC8D4AD3778A4B8C4A5A608C4A9A6023
:106140008C4ADA608C4A1A61FFF7E8F96068E378F4
:106150000002184306D4824B5B689847824B586113
:10616000FFF7DCF97F4B04221A70FFF7D7F962685A
:10617000E37812021A437C4B9A62804B9B7E012B80
:1061800001D0FFF7CBF9FDF7E7F9FFF7C7F9E278A0
:10619000754B1A76FFF7C2F96268E37812021A4368
:1061A000714B1A62754B9B7E012B01D0FFF7B6F93C
:1061B000E9E76168E378090219430129D2D8C9B235
:1061C0000020FDF76DFFFFF7A9F96268E37812027E
:1061D0001A43654B5A62694B9B7E012B01D0FFF736
:1061E0009DF9D0E76168E3780A021343022BB9D81E
:1061F000FEF7BEFA002801D100F0A4FCFEF7B8FAC1
:106200000E2801D100F09EFC564B04221A70FFF7B5
:1062100085F96168E378090219430129A2D8C9B256
:106220000020FDF727FFFFF779F96168E37809029D
:106230001943032996D8C9B20020FDF747FFFFF79D
:106240006DF94F4A012313706068000201D500F018
:10625000C1FC002201930092002020210023FDF7C1
:1062600033FA6068E37800021843C1173C4B4018CA
:1062700048405B68A57898472721021C281CFDF739
:106280005BFAFFF74BF96268E3781002184301D517
:10629000FFF744F9344BDB7F012B01D0FDF7A8FF5A
:1062A000011E00D1DBE3374801F08CFBA478021C0F
:1062B0001321201CFDF740FAFFF730F96168E378FD
:1062C0000802184300D54DE7274BDB7F012B01D097
:1062D000FDF78EFF011E01D100F00EFC294801F0F0
:1062E00071FBA478021C1421201CFDF725FAFFF78E
:1062F00015F96168E3780802184300D532E71A4BB4
:10630000DB7F012B01D0FDF773FF011E00D1ADE350
:106310001C4801F057FBA478021C1521201CFDF736
:106320000BFAFFF7FBF86368E2781B021343012BBB
:1063300000D917E70A4A1370FFF7F0F80F4B094C22
:106340009B7E6360FFF7DCF8074B064C1B7E6360A7
:10635000FFF7D6F8044B034C1B6A6360FFF7D0F8D5
:106360008CF0FF1F0CF4FF1FB8F0FF1F95410000D9
:10637000F1410000D141000031420000F4F0FF1F64
:1063800018F1FF1F80969800F74BF84C9B6A6360EA
:10639000FFF7B6F8F44BF54C5B6A6360FFF7B0F8B3
:1063A0006068E37800021843FEF74EFFFFF7B6F887
:1063B0006068E37800021843FEF710FFFFF7AEF8BD
:1063C0006068E37800021843FEF714FFFFF7A6F8B1
:1063D0006068E37800021843E54BDB6898472821A2
:1063E000021C0020FDF7A8F9FFF798F81021002003
:1063F000FDF7B2F9E178021C130CD2B2A078DBB23F
:106400000091019210210022FDF75EF9FFF786F856
:106410006268E37812021A4300202D21FDF78CF9FF
:10642000FFF77CF86268E37812021A43002021210A
:10643000FDF782F9FFF772F86068E378000218430D
:1064400003F0A4FAC74BC64A02F048F803F088FCF0
:1064500003F068FA1121021C0020FDF76DF9FFF727
:106460005DF838210020FDF777F98023DB00021C5E
:1064700061681A40E37809021943BE4BA0780B40CB
:106480001A433821FDF758F9FFF748F8E178002062
:10649000FDF7DCFDFFF742F8E1780020FDF73CFE58
:1064A000FFF73CF86068E37800021843C117B04B6F
:1064B00040185B6848409847AB4BD860FFF72EF810
:1064C000E1780020FDF708FCFFF728F86068E37822
:1064D00000021843C217A64B80185B6850409847CB
:1064E000A14B1861FFF71AF834210020FDF734F9A9
:1064F000031C6068E27801020A43A078002A00D1F8
:1065000088E3802212011A433421FDF715F9FFF7C1
:1065100005F86068E37800021843FEF78FFEFEF787
:10652000FDFFE1780020FDF719FCFEF7F7FFE178A9
:106530000020FDF7DFFD0021A078FDF70DF9021C1A
:106540006068E37801021943A0780423002900D190
:10655000F3E21A430021FDF7EFF8FEF7DFFF606872
:10656000E37800021843FDF7A7F8FEF7D7FF60684D
:10657000E378000218437E4B5B6898472521021C94
:106580000020FDF7D9F8FEF7C9FF6068E378000244
:106590001843774BDB6898472421021C0020FDF745
:1065A000CBF8FEF7BBFFE1780020FDF7ABFBFEF771
:1065B000B5FF6068E37800021843FEF721FEFEF79E
:1065C000ADFFE1780020FDF733FBFEF7A7FFE3788E
:1065D0000821C91AC9B20020FDF79EFA664B9B7EBE
:1065E000012B01D0FEF79AFFCDE56068E378000249
:1065F0001843FEF717FEFEF791FF6068E37800028C
:106600001843FEF7F1FDFEF789FF6068E3780002AA
:106610001843FEF7FBFDFEF781FF34210020FDF754
:106620009BF8021C6068E37801020B43A078002B02
:1066300000D08EE201231A433421FDF77DF8FEF7E6
:106640006DFF6268E37810021843494BDB68984796
:106650004A4B012118604A4B021C1970A078262170
:10666000FDF76AF8FEF75AFF10210020FDF774F8D5
:10667000021C110AC9B2D2B2A078E378009101924B
:1066800010210022FDF720F8FEF748FF34210020FA
:10669000FDF762F8021C6068E37801020B43A07802
:1066A000002B00D1C4E204231A433421FDF744F83F
:1066B000FEF734FF0020FDF7D7FB002800D04FE2A3
:1066C000A078E178FDF7A0FAFEF728FF6068E3788C
:1066D00000021843FEF7ACFDFEF720FF0020FDF797
:1066E000C3FB002800D0AAE2A078E178FDF77AFA8F
:1066F000FEF714FF34210020FDF72EF8021C60681D
:10670000E37801020B43A078002B00D09DE2022326
:106710001A433421FDF710F8FEF700FFE17800205E
:10672000FDF7C4FAFEF7FAFE6068E378000218434A
:106730000F4B5B6898472B21021C0020FCF7FCFFE5
:10674000FEF7ECFE6068E37800021843084B5B68D4
:1067500098473321021C0020FCF7EEFFFEF7DEFE17
:1067600073989E1FB5F80440B8F0FF1F0CF4FF1F8C
:106770008CF0FF1FFFFBFFFFF4F0FF1F1CF3FF1F58
:1067800020F3FF1F6068E37800021843F74BDB68D3
:1067900098472A21021C0020FCF7CEFFFEF7BEFE20
:1067A0006068E37800021843F04B5B689847232148
:1067B000021C0020FCF7C0FFFEF7B0FEE1780020CD
:1067C000FDF7DAFBFEF7AAFE34210020FCF7C4FF38
:1067D000021C6068E37801020B43A078002B00D113
:1067E0001FE208231A433421FCF7A6FFFEF796FEAA
:1067F0006068E37800021843FEF70EFDFEF78EFE98
:10680000E1780020FDF794FAFEF788FE6268E378ED
:1068100010021843C317C0185840D44B5B68984700
:10682000D34DD44B012228601A702021A078FCF7A8
:1068300093FF410701D4FEF771FEA0782A68272153
:10684000FCF77AFFFEF76AFE34210020FCF784FF94
:10685000021C6068E37801020B43A078002B00D192
:106860009CE110231A433421FCF766FFFEF756FE25
:1068700010210020FCF770FF021C130C120AD2B288
:10688000A0780092E278DBB2019210210022FCF79E
:106890001BFFFEF743FEE1780020FDF793F9FEF7BA
:1068A0003DFEE1780020FDF731FBFEF737FEE17891
:1068B0000020FDF705FBFEF731FEE1780020FDF733
:1068C00011FBFEF72BFE6268E37812021A430020E8
:1068D0001121FCF731FFFEF721FEE1780020FDF7E2
:1068E00039FBFEF71BFEE1780020FDF75BFBFEF7AE
:1068F00015FEE1780020FDF71DFBFEF70FFEE178A5
:106900000020FDF7A9F9FEF709FEE1780020FDF768
:10691000B7F9FEF703FEE1780020FDF735F9FEF741
:10692000FDFD0020FDF746F9934C6060FEF7E8FDA1
:1069300000201021FCF710FF8F4CC0B26060FEF702
:10694000DFFD0020FDF7FCF88B4C0823181A60606F
:10695000FEF7D6FD00201021FCF7FEFE864C031446
:10696000DBB26360FEF7CCFD814B1868FFF799F846
:10697000824BD868FFF795F800201021FCF7ECFE59
:106980007D4C0312DBB26360FEF7BAFD00202D21BF
:10699000FCF7E2FE784C6060FEF7B2FD774B1869B9
:1069A000FFF77FF8764B1868704B1B699847724C5D
:1069B0006060FEF7A5FD10210020FCF7CDFE6F4CB6
:1069C000C104C90E59206176FCF7C0FC627E6A4B97
:1069D0005A60FEF7A3FD6B4C5020211C0422FCF7EB
:1069E000D9FC624B20689B689847634B5860FEF760
:1069F00095FD634B1868FDF71BFC604C042260603A
:106A0000211D4420FCF7C6FCE37F002B00D146E1AA
:106A10006268594B5A60FEF781FD554B1868FDF7C7
:106A2000E7FB564C04222060211C4020FCF7B2FCFE
:106A3000E37F002B00D12BE122684F4B5A60FEF719
:106A40006DFD514C4C20211C0422FCF7A3FC474B4C
:106A500020689B689847484B5860FEF75FFDA07818
:106A600013214A4AFCF768FEFEF758FDA07815216D
:106A7000464AFCF761FEFEF751FD10210020FCF7AD
:106A80006BFE1F233D4C011C19405A20A176FCF7D8
:106A90005DFCA27E384B5A60FEF740FD10210020BD
:106AA000FCF75AFE354C0103090F5B20E176FCF739
:106AB0004DFCE27E304B5A60FEF730FD0020FDF7C2
:106AC00079F82E4C011C20775C20FCF73FFC227FDC
:106AD000294B5A60FEF722FD0020FDF731F808210E
:106AE000264C091AC9B25D206177FCF72FFC627F42
:106AF000214B5A60FEF712FDA0781421234AFCF7BF
:106B00001BFEFEF70BFD1C4B04221A70FEF706FD60
:106B10001A4AD377154B1E4A5A609A60DA601A6196
:106B2000FEF7FCFC1B4C04226420211CFCF732FC09
:106B30002268114B5A60FEF7F1FC9A43FCF7FCFD0A
:106B4000FEF7ECFCE278144B9A76FBF7C5FFFEF7F4
:106B5000E5FC01239A433421FCF7EEFDFEF7DEFC51
:106B6000A078E178FDF710F9FEF7D8FC8CF0FF1F54
:106B700024F3FF1F18F1FF1F0CF4FF1FB8F0FF1FD5
:106B80001CF3FF1FC8F0FF1FC4F0FF1FFFFF0F0023
:106B900059420000DCF0FF1FF4F0FF1F10239A435E
:106BA0003421FCF7C9FDFEF7B9FC404C1A20A17E48
:106BB000FCF7CCFBA27E3E4B5A60FEF7AFFC3D4C8F
:106BC00004226820211CFCF7E5FB2268384B5A6040
:106BD000FEF7A4FC0023022201920093181C20213E
:106BE0001A1CFCF771FDFFF73CFB334C5820217E4B
:106BF000FCF7ACFB227E2E4B5A60FEF78FFC2F4C2D
:106C000004226020211CFCF7C5FB2268284B5A6037
:106C1000FEF784FC2A4A34211A40FCF78DFDFEF76A
:106C20007DFC08239A433421FCF786FDFEF776FCB1
:106C300004239A433421FCF77FFDFEF76FFCA07814
:106C4000E178FDF7BDF8FEF769FC02239A43342191
:106C5000FCF772FDFEF762FC5868FDF7B9FA144BB9
:106C60005860FEF75BFCA078FDF722F9104C6060DD
:106C7000FEF746FCA078FDF70FF90D4C6060FEF7BB
:106C80003FFC1868FDF786FA094B5860FEF746FC92
:106C90002068FDF77FFA064B5860FEF73FFC6068FE
:106CA000FDF796FA024B5860FEF738FCF4F0FF1F30
:106CB0000CF4FF1FE0F0FF1FB8F0FF1FD8F0FF1F1C
:106CC000FFF7FFFF38B5B34CA378002B23D16378CF
:106CD000552B00D18AE034D8472B00D12DE15ED965
:106CE0004D2B00D1DFE000D8CEE0512B00D192E057
:106CF000542B00D076E00A2800D130E1092809D1D0
:106D00006268E37812021A43012A00D89EE1A24B7E
:106D100004221A7038BD022B2AD09F4B04221A700D
:106D20000A28F7D19D4A1278002AF3D05B689C4A62
:106D30001360002B50D09B4B0822196891431960B7
:106D4000E8E7832B00D1D9E039D9852B00D1EAE0DF
:106D500000D2B5E0F02B00D186E0FF2B42D10A280B
:106D600000D110E10928D5D1E2788F4B1A70D1E714
:106D70006278372A36D80A2800D1EAE009287BD081
:106D80000B2800D14EE10C28C4D1101C874B920077
:106D9000A030D11880000422FCF7E8FABAE7452BAE
:106DA00000D197E04BD8402B1CD10A2800D143E1F9
:106DB0000928AFD1E1787E48FCF7C8FAAAE7812B11
:106DC00000D1A5E048D8802B0CD10A28A2D1794A5D
:106DD000714B12785A60A5E7724B082219680A4372
:106DE0001A6097E76C4B03221A7099E70A2800D1C2
:106DF000FDE0092800D08DE76268E37812021A43AB
:106E0000012A00D983E76C4919204B7601221931F8
:106E1000FCF7C0FA7EE70A2800D1AAE0092800D0D2
:106E200078E7654D0123EA7DE178134202D00B42F9
:106E300000D107E11720E975FCF788FA6AE70A280C
:106E400000D191E0092800D064E7E1785A4B08208E
:106E50009960FCF77BFA5DE70A2800D05AE7574AA9
:106E60004D4B12685A605DE70A2800D052E7544A39
:106E7000494B12785A6055E76168E3780902194373
:106E80004A4B9200D15045E7482BABD10A2800D19C
:106E9000A3E0092800D03DE7E178474B0C20D960FA
:106EA000FCF754FA36E70A2800D19BE0092800D005
:106EB00030E7E178404B16209975FCF747FA29E74F
:106EC0000A285BD0092800D024E7334B5A683D4B91
:106ED0001A601FE70A2800D19AE0092800D019E7B4
:106EE0006368E1781B020B43023B062B00D90EE7D7
:106EF000314B02209970FCF729FA0BE70A2867D07A
:106F0000092800D006E7244B5A682F4B1A6001E786
:106F10000A2800D0FEE6274A1F4B1278043A514255
:106F20004A415A60FEE60A2866D0092800D0F1E6F8
:106F3000194B5A68254B1A60ECE60A286DD00928CF
:106F400000D0E7E6E1781C4B04205960FCF7FEF91D
:106F5000E0E616499200104B52585A60E2E6164A93
:106F60000D4B127E5A60DDE6134A0B4B92685A6055
:106F7000D8E6114A084BD27D5A60D3E6114B1A6805
:106F8000054B5A60CEE6084A034B1278511E8A41DF
:106F90005A60C7E630F3FF1F0CF4FF1FF5F3FF1F25
:106FA00090F3FF1F38F3FF1FF4F3FF1F20F4FF1FC0
:106FB000FF070000FCF3FF1FF4F0FF1FC4F3FF1FE7
:106FC000F0F0FF1FF8F3FF1F20F8FF1F18F4FF1F5A
:106FD000224A234B12685A60A4E6224A204BD26808
:106FE0005A609FE61F4A1E4B927D5A609AE61D4AE0
:106FF0001B4B527E5A6095E61B4B1C4A19684A434C
:107000001B4952181A60164B520052085A6089E602
:10701000144A134B92785A6084E6124A104B526815
:107020005A607FE6101C134B9200A030D1188000EC
:107030000422FCF7AFF96DE60F48FCF773F9084B33
:1070400058606FE6FCF726FAE178F3E60549182068
:107050000B7601221831FCF79DF95BE620F8FF1F43
:107060000CF4FF1FF4F0FF1F18F4FF1F6D4EC64114
:107070003930000020F4FF1FFF07000008B50A4B5D
:107080009A78022A09D15868DA7801020A435878B6
:10709000002A06D1FBF7DCFD02E0044B04221A7043
:1070A00008BDFBF7D7FDFBE730F3FF1F0CF4FF1F14
:1070B00008B5194A9378012B21D0002B19D0022B47
:1070C00011D0164B04221A70154A1278002A09D0E2
:1070D0005B68144A1360002B17D0134B0822196801
:1070E0009143196008BD5078FBF7B0FD0B4B586019
:1070F000EAE75078FBF77EFD084B5860E4E75078EC
:10710000FBF7AAFD054B5860DEE7074B082219681C
:107110000A431A60E6E7C04630F3FF1F0CF4FF1F76
:10712000F5F3FF1F90F3FF1F38F3FF1F08B5054B62
:107130005A68D8781202024359780020FCF7FCFA0A
:1071400008BDC04630F3FF1F08B5044B0020597836
:10715000FCF702FB024B586008BDC04630F3FF1F2E
:107160000CF4FF1F10B5002384B0644C01936378C6
:10717000142B00D99FE0624A9B00D3589F46FCF72E
:10718000DBF904B010BD6068E3780002184380B2F8
:10719000FCF7C8F85B4B5860F3E76168E3780802D6
:1071A000184380B2A178FCF7D1F8A278554B5A6009
:1071B000E7E76068E37800021843042280B201A97F
:1071C000FCF7D4F84F4B019A5A60DAE76068E3782D
:1071D00000021843019080B201A90422FCF7DAF8FA
:1071E000484B01995960CCE7A078802212018018A1
:1071F00001A90422FCF7BAF8424B01995960C0E793
:107200006168E3780A0213430193A0788022120197
:107210008018E1E7A078802212018018FCF782F83C
:10722000384B5860ADE7002037491C22FCF7B2F814
:10723000A7E7402035492C22FCF7ACF8A1E7FCF782
:1072400029F99EE76368E27818021043304A9042B9
:107250003FDD012252421B0EE2701B060722134340
:107260002C48636002AC211CFCF7D6F86268E37816
:1072700012021A43234B5A6083E76368E2781802CC
:107280001043234A90421ADC80B202A9FCF7C4F8EA
:10729000A378002B1FD0012B26D0022B29D0DA1E79
:1072A000032A1DD802A9CA5C164B5A6069E7154B20
:1072B00007225A6065E7134B03221A7061E7012227
:1072C00052421B0EE2701B060722134363601148F3
:1072D000DBE780B2C6E76B461A7A0A4B5A6050E782
:1072E000084B04221A704CE769464A7A054B5A60EB
:1072F00047E76B469A7A034B5A6042E730F3FF1F29
:1073000068A500000CF4FF1FF4F0FF1FB8F0FF1F8A
:10731000FE070000FF0700007047C0467047C046E8
:1073200008B50F4B5B78012B14D0002B0AD0022B31
:1073300003D00C4B03221A7008BDFDF719FA094B54
:107340005860F9E7084B9B7E002B06D0054B0422C2
:107350001A70F1E7FDF702FAEEE7FDF7F5F9EBE752
:1073600030F3FF1F0CF4FF1FF4F0FF1F08B5064BAE
:107370005868DA78054B000210435B689847404232
:10738000FCF7D6FA08BDC04630F3FF1F8CF0FF1F94
:1073900008B5054B5868DA78044B000210435B6867
:1073A0009847FCF7C5FA08BD30F3FF1F8CF0FF1FAC
:1073B00008B5FCF7FDFA08BD10B5304CA378002BDA
:1073C00014D16278012A19D0002A2BD0022A11D1B7
:1073D0002B4A13702B4A13706368E2781B02134325
:1073E000142B3DD9284B09221A7002E0264B0422A7
:1073F0001A7010BD244B03221A70FAE7204A13704A
:10740000204A1370214B1B78012B18D0002B2FD052
:10741000022B23D11E4B9B7E012B10D1FCF746F98A
:10742000021C11E0164B1A70164B1A706068E37854
:1074300000021843174B1968FCF7F6FAD9E7002049
:107440002121FCF789F9021C6168E3780902081C14
:107450001843104B1968FCF719FBCAE70022F3E741
:107460000D4A9B0098580B4B1968FCF7DDFAC0E7F2
:1074700000202D21FCF770F9021CE5E730F3FF1F17
:10748000B4F0FF1FE4F0FF1F0CF4FF1F8CF0FF1F90
:10749000F4F0FF1F24F3FF1F3CF3FF1F194B5B7831
:1074A000002B11D1184B01221A70184B18485B7829
:1074B0000370184B1A68431C093011780132197097
:1074C00001338342F9D17047012B12D0022BFAD13C
:1074D0000D4B01221A700D4B0D495B780E480B7055
:1074E00000230133C218093A1278CA54082BF8D184
:1074F000E9E70A4A0421D1715371F6210023917101
:107500001371E0E730F3FF1F94F3FF1FF4F0FF1F48
:1075100098F3FF1F0CF0FF1F002000000CF4FF1F6A
:107520000249034B034AD1507047C0460400FA0594
:107530000C0D000000E000E008B5164B5A78812AD7
:1075400003D0154B04221A7008BD9A78922AF8D1FC
:107550009A79A32AF5D15A79B42AF2D11A79C52A8F
:10756000EFD1DB78D62BECD1FBF720FB72B6FBF723
:107570001FFC0A4B0122524280215A50C02149006F
:107580005A50074A074B08491A60084B084AD1501D
:10759000DAE7C04630F3FF1F0CF4FF1F00E100E004
:1075A0007856341200F0FF1F0400FA050C0D00009D
:1075B00000E000E038B54F4B4F4C18786422227041
:1075C00060705D68DA7829024C4D0A438100695881
:1075D00062608F464A4B9A4202D14A4B01221A708E
:1075E00038BDFFF7A9FFFBE759780020FCF7B4F896
:1075F0006060F5E759780020FCF79EF8F0E7FDF7AA
:1076000041F9EDE7FDF748FCEAE7FDF70FFBE7E797
:10761000FFF744FFE4E7FDF725FBE1E73A4B587835
:10762000D97DFDF7E1FBDBE7FDF7FAFAFBF7BCFAE2
:10763000D6E7FBF7BBFA344BD87DFDF7CFFACFE79F
:10764000FDF7FCF8CCE7FDF7F3F8C9E7FDF7DCF848
:10765000C6E7FDF711F9C3E7FFF784FDC0E7FDF7C3
:10766000A1F8BDE7FDF752FABAE7FDF7B9F8B7E7B9
:10767000FDF784F8B4E7FDF7D9F9B1E7FDF746FD6A
:10768000AEE7FDF70BFDABE7FDF7EAFCA8E7FDF77A
:1076900033FCA5E7FDF768FCA2E7FDF7EBFB9FE7EE
:1076A000FDF788FB9CE7FDF721FB99E7FDF72AFB37
:1076B00096E7FDF75FFA93E7FDF742F990E7FFF7EA
:1076C000F7FC8DE7FFF72CFE8AE7FFF7FBFA87E769
:1076D000FDF706FF84E7FFF76FFE81E7FCF768F927
:1076E0007EE7FFF743FE7BE7FFF752FE78E70223D2
:1076F000237075E730F3FF1F0CF4FF1FBCA50000DB
:10770000D204000050F8FF1FF4F0FF1FF0B5824BC9
:1077100085B01B78071C002B4ED0804B1B78062BA6
:107720004AD00A2B48D0102293430F2B44D07C4DD3
:107730007C4E00232B7533707B4B6C461B78002BE3
:1077400049D16846FBF7BAFB00284DD1774C217828
:107750004B1E012B00D896E02B7D0422181C904371
:10776000021C042900D180E0002A23D0082B21D05C
:10777000062B1FD0FFF71EFF2B7D092B1AD1237874
:10778000022B00D19FE06A4B1D68002D12D0237898
:10779000012B0FD1674B68481968026800238A42A1
:1077A00005D1A8E09A0082588A4200D1A3E00133B3
:1077B000AB42F7D105B0F0BD594D6C462B7D013B76
:1077C000DAB2012A39D9574E00232B753370564B44
:1077D0001B78002BB5D05949594B5A4A6846D150AD
:1077E000FBF76CFB0028B1D0227A4C4B1A70627AFE
:1077F0005A70A27A9A70E27A9A71227B5A71627BED
:107800001A71A27BDA7062784F4B1A70FBF7D6FAC6
:107810004E4B002218604E4B1A702378072B4BD02A
:1078200002232B75414C21784B1E012B47D905298A
:1078300045D0484B01221A708EE75A1E93410733F8
:107840002370414B4449374E1B7888683278637007
:1078500000230190A370002A1DD0012A36D068466B
:10786000FBF786FB0028A5D0AEE72C4909787F29D5
:1078700000D979E7002A9DD0082B9BD0062B99D000
:10788000FDF740FB96E7012F29D02B7D0422181C21
:107890009043021C68E74B682372304B1978617281
:1078A0005978A172D979E172997921735979617303
:1078B0001B79E273A373D2E701232B75B2E7254B43
:1078C00000221A7048E7052323705CE72448002350
:1078D0000133C15CE218D171082BF9D1BFE7154A19
:1078E000204913688B4209D92B7D0422191C91432E
:1078F00020700A1C38E7052323705BE7591C1160D0
:1079000098B20649FBF788FD09232B75114B2178A6
:107910001F700922092324E7F4F3FF1F30F3FF1F30
:107920008CF0FF1F94F3FF1F50F8FF1FFCF3FF1FA5
:1079300000F4FF1FC4F3FF1FC8F3FF1F0400FA0584
:107940000C0D000000E000E051F8FF1FECF0FF1FFD
:10795000ACF0FF1FF5F3FF1FF4F0FF1F0CF4FF1F47
:1079600098F3FF1FFE070000054B5A68D978054BB6
:1079700012020A439A4202D1034B01221A70704745
:1079800030F3FF1FD204000050F8FF1FC046C0466E
:1079900038B5FBF713FA0A4C051C2368C21AFA2300
:1079A0005B009A4208D86268AB1A322B03D90020D8
:1079B000FBF760F8656038BDFBF7D6F82560F2E7A5
:1079C000A4F0FF1F002934D00123002210B4884204
:1079D0002CD301242407A14204D2814202D20901FE
:1079E0001B01F8E7E400A14204D2814202D249001F
:1079F0005B00F8E7884201D3401A1A434C08A042C2
:107A000002D3001B5C0822438C08A04202D3001B57
:107A10009C082243CC08A04202D3001BDC0822436E
:107A2000002803D01B0901D00909E3E7101C10BC92
:107A30007047002801D00020C04307B4024802A1CB
:107A40004018029003BDC046D90000000029F0D0C4
:107A500003B5FFF7B9FF0EBC4243891A1847C04669
:107A6000002941D010B4041C4C40A446012300223C
:107A7000002900D54942002800D5404288422CD335
:107A800001242407A14204D2814202D209011B0130
:107A9000F8E7E400A14204D2814202D249005B002F
:107AA000F8E7884201D3401A1A434C08A04202D397
:107AB000001B5C0822438C08A04202D3001B9C08D8
:107AC0002243CC08A04202D3001BDC08224300283A
:107AD00003D01B0901D00909E3E7101C6446002C00
:107AE00000D5404210BC7047002806D003DB0020C0
:107AF000C043400801E08020000607B4024802A10C
:107B00004018029003BDC046190000000029EBD0C8
:107B100003B5FFF7A7FF0EBC4243891A1847C046BA
:107B20007047C0468446101C62468C46191C63464A
:107B300000E0C0461FB501F0BDF8002801D40021C7
:107B4000C8421FBD10B500F0EDFF4042013010BD2E
:107B500010B501F0AFF8002801DB002010BD0120B6
:107B600010BDC04610B501F0A5F8002801DD0020C9
:107B700010BD012010BDC04610B501F01DF8002851
:107B800001DC002010BD012010BDC04610B501F081
:107B900013F8002801DA002010BD012010BDC046F6
:107BA000F0B55F4656464D464446F0B446024500A1
:107BB000C00F85B00F1C760A2D0E804641D0FF2DD8
:107BC00026D08024240400212643F6007F3D8946E8
:107BD0008B46F90F7C027800640A000E00918A46F9
:107BE0003CD0FF2834D080231B041C430023E40036
:107BF0007F380193009F4346019A7B4049469C464B
:107C000011430F2900D971E0764F89007F58BF4694
:107C1000002E3ED10822022391469B46D9E75A46C0
:107C2000341CC24601920199022937D0032900D1A0
:107C3000CFE0012900D0ABE053460B4000220026E4
:107C400032E0002E19D10421012289469346C0E773
:107C5000221C531E9A4102320192CBE70127019761
:107C6000002CC7D0201C01F021FF431F9C4076232D
:107C70005B420021181A0191BCE7301C01F016FF8D
:107C80007625431F9E406D4200232D1A99469B4640
:107C90009FE70C23032199468B469AE7D44601239C
:107CA00067463B40FF2200267602D205700ADB07BA
:107CB0001043184305B03CBC90469946A246AB46DB
:107CC000F0BD80260023F603FF22EDE70022002608
:107CD000EAE78020C00306423BD0044239D1061CAB
:107CE00026437602760A009BFF22DDE7281A0390DE
:107CF00076016401A64239D3361B1A2201230120E2
:107D0000311C5B007600002901DBB44201D8361B30
:107D10000343013A002AF3DC741EA641341C1C43C1
:107D2000039A7F32002A27DD630704D00F23234004
:107D3000042B00D00434270103D52B4B039A1C409D
:107D40008032FE2A0BDD012361460B40FF22002614
:107D5000AAE706437602760A4346FF22A4E7A40177
:107D600001236746660AD2B23B409DE7039F1B2270
:107D7000013F03970023C2E77E23039F5B42DB1B87
:107D80001B2B07DD012361460B40002200268BE7F9
:107D9000D446C5E7221CDA40039B9E339C40231C3B
:107DA0005C1EA34113435A0704D00F221A40042A31
:107DB00000D004335F0105D5012361460B40012249
:107DC000002671E79E01624601231340760A0022D5
:107DD0006AE78026F60326437602760A5346FF2298
:107DE00062E7C046BCA90000FFFFFFF770B5041EA4
:107DF0003CD0C60F00D04442201C01F057FE9E2309
:107E0000251C1B1A962B0CDC083884406402640A7B
:107E1000DBB2321C6402DB05600AD2071843104350
:107E200070BD992B0ADD0522121A211CD1400A1CB3
:107E3000011C1B318D40691E8D411543052801DD54
:107E4000421F9540164C2C406A0704D00F22154063
:107E5000042D00D0043461010CD59F23181AFF288B
:107E60001AD0A401640AC3B2321CD3E70022002353
:107E70000024CFE7E408FF2B04D06402640ADBB2DD
:107E8000321CC7E7002C04D08020C00304436402E6
:107E9000640A321CFF23BDE7321CFF230024B9E72C
:107EA000FFFFFFFBF8B55F46564644464D46F0B42B
:107EB0000C034D00CE0F610A440F2143C400180388
:107EC00080465800400D8246D80F84464046400AFE
:107ED000530F0343D0006D0D371C83465246664551
:107EE00000D19DE0AF1A002F00DC03E1002A38D159
:107EF000184300D0E4E0630709D00F232340042B8C
:107F000005D0231DA342A441644209191C1C080288
:107F100000D478E0CE4B6A1C9A4200D105E1CD4BEB
:107F2000E408194048075205490204430B0B520D5F
:107F3000371C002000211B03201C1C0B0B0D1B05F4
:107F4000C54D2343520552081D4015436D006D0871
:107F5000FF07291C39433CBC90469946A246AB46D4
:107F6000F8BDBB488542C6D0802000040343382FAB
:107F700000DDECE01F2F00DD20E12020C01B1A1CDB
:107F8000814682405846F8400243944658464A4645
:107F90009040421E9041FB40624602431F1CA21AC1
:107FA0009442A4416442C91B091B141C0B02A2D5B4
:107FB00049024F0A002F00D1C4E0381C01F076FDC1
:107FC000021C083A1F2A00DDB7E02821091A201CEC
:107FD0009740C84007439440954200DDA9E0551BF7
:107FE000691C1F2900DDD8E01F22551B3B1C221CE9
:107FF000AB40CA40AC40651EAC411343CF401C436C
:10800000391C002577E74807E4086A05C908520DBE
:10801000371C04438E4B9D4248D009030B0B88E765
:10802000AA1A9446002A00DC98E05046002853D053
:108030008748854200D15EE7802000040343624602
:10804000382A00DDFDE01F2A00DD4BE120226046DA
:10805000101A1A1C82408246914658466246D04009
:108060004A4602439046584652469040421E90412E
:10807000424602436046C3401219A242A4416442F0
:1080800059180919141C080200D434E7704B013543
:108090009D4200D124E16F4B600819400123234029
:1080A0001C1C0443CB071C43490824E70B1C234337
:1080B00000D1C7E180231B030B431B031B0B38E7D5
:1080C000013F002F64D15846221A9442A4416442D1
:1080D000C91A091B141C69E75846184300D10AE75E
:1080E0000122524294446046002800D0C5E0584620
:1080F0000219C2E7002F72D1681C4005400D01280B
:1081000000DCDEE05A46A21A9442BF41C81A7F4200
:10811000C71B380200D488E05A46141BA34592417D
:10812000591A52428F1A664644E7371C002300242E
:10813000FFE64849AD1A3940DDE6271C283887405C
:10814000002449E7201C01F0B1FC203038E75A46F2
:108150001A43531E9A41D2B2002720E7002A00D0CA
:10816000DDE0681C4205520D012A00DC8EE0384D2E
:10817000A84200D1B3E05D462A19A242A44164425C
:1081800059180919CC07520814434908051CB2E6CE
:108190002F48854200D0EAE6ADE62B1C1F3B3A1C77
:1081A000DA40131C20296DD03F22551BAF403C43C1
:1081B000601E84411C43002100259CE6381C2038A9
:1081C0001A1CC240101C202F5ED04022D71BBB407F
:1081D0005A461A43531E9A4102430027DFE6002DF8
:1081E0003CD01B4DAA4500D194E080252D047F4250
:1081F0002943382F00DDADE01F2F00DD2CE12025C5
:10820000ED1B081C261CA840FE40AC400643651E22
:10821000AC413443F9405D462C1BA34592415B1AA7
:108220005242991A55466646C0E6131C3B43141C3D
:10823000002B00D0BEE600270022002500210024EC
:10824000E8E65A461A43531E9A41D2B2002313E776
:10825000FF070000FFFF7FFFFFFF0F800D1C25437E
:1082600058D0FF43002F51D1041BA3459241591A06
:108270005242891A5546664698E69648854200D08D
:10828000DDE638E6002792E70023A1E7081C20433B
:10829000002D00D0C0E0002800D1FBE05846184374
:1082A00000D128E658460219A242A4416442591856
:1082B0000919141C0A0200D41DE6874B0125194038
:1082C00019E6081C2043002D39D100286DD15946EC
:1082D000194300D1BDE0191C5C4666460BE6051C3F
:1082E0002A1CABE7604620381A1CC2406046914603
:1082F000202800D1ABE04022121A93405A461A437C
:10830000531E9A414B461A430023B5E6714DAA45C8
:1083100000D06EE7191C5C4655466646EBE5002D1D
:108320001ED10D1C254373D0D543002D6DD15C4467
:108330005C4592415918524289185546A3E60028D7
:1083400049D15946194300D196E0191C5C4666464E
:10835000604DD0E50C43611E8C41E4B200215AE728
:108360005C4DAA4554D05542802210040143382D5B
:1083700000DD85E01F2D00DD95E02022501B0A1C4A
:1083800084468240201CE840024390466246944066
:10839000601E844142461443E9405C445C4592417E
:1083A000CB185242991855466DE65846184300D1ED
:1083B000A1E55846271ABC429241C81A5242801A77
:1083C00002026AD55846041BA3459241591A5242EB
:1083D000891A66468FE55846184336D04807E408A0
:1083E00004438020C9080003014208D0DD0805428B
:1083F00005D15946CA085C071443291C6646630F19
:10840000C9001943E400334D75E5324A9245AED1B7
:10841000191C5C4655466EE5002837D0584618436F
:1084200013D080254807E408C9082D0304432942D6
:10843000E5D0D8082842E2D15D46EA085C0714433B
:10844000011CDCE70023002473E5224D53E50023E3
:1084500054E700270022F1E63D1C203D0A1CEA40BB
:10846000151C202F31D04026F71BB9400C43611E4C
:108470008C412C430021CEE6164A0027151CDDE670
:108480000C43611E8C41E4B2002186E7191C5C4656
:10849000104D30E5191C5C462DE5031C3B43D8D03C
:1084A000011C3C1C27E52020404240190A1CC24008
:1084B0009046202D0BD04020451BA9400C43611E47
:1084C0008C4145462C43002167E70021CEE700217F
:1084D000F4E7C046FF070000FFFF7FFFF0B55646F8
:1084E00044465F464D46F0B41F1C0B031B0B9846D9
:1084F0004B0087B0041C81465B0DC80F161C9A46C2
:108500000090002B51D06A4B9A4531D080224146D1
:1085100052030A43630FD2001A43664B904600256C
:10852000E20091469A44002402953B031B0B9B46B4
:10853000FD0F7B00311C5B0D019560D05C4A9342BE
:1085400054D08021584649030143720FC90011439A
:10855000584A8B469B18F1000020009A04436A4059
:1085600003920F2C00D9ADE0534EA4003459A74616
:10857000404604436ED100210225082488468946DE
:108580000295D2E7009C0298C3464946019402280E
:1085900064D0032800D1ABE2012800D038E2019A70
:1085A000002402400025A14660E0434623434AD010
:1085B0004046002800D1C0E101F078FA031E272BC5
:1085C00000DDB3E128210D1A211C083B4246E94099
:1085D0009A400D1C1543221C9A40A8469146374BE1
:1085E00000251B1A9A46002402959EE75A46164318
:1085F0000320002EB1D1B34600210220ADE75A4638
:1086000032431BD05B46002B00D18AE1584601F073
:108610004DFA272800DD7DE12822171A011C321CA3
:1086200008395B46FA408B40171C1F43331C8B40B4
:10863000BB46191C214B1B1A00208EE70027BB46A6
:108640000021012089E7002001250424804681467D
:1086500002956AE703250C24029566E7019C0394C2
:10866000039D01222A400024114DA1460020002133
:108670002403260B0C0D2405114B34432D052340F8
:108680002B435B005B08D207191C4846114307B017
:108690003CBC90469946A246AB46F0BD00228024E1
:1086A00024039146024DE1E700240025A146DDE7C1
:1086B000FF07000001FCFFFFFCA900000DFCFFFF0D
:1086C000FFFF0F805546ED1A0495D84500D953E1B8
:1086D00000D14EE1049C0025013C4E4604944746DF
:1086E000A946584603020C0E1C430902250C23041C
:1086F0001B0C0091381C291C0193FFF763F90199A9
:1087000083464143381C8A46291CFFF79FF9330CE6
:10871000090419438A450CD95B460919013B8C426F
:1087200000D947E18A4500D844E1022252429344ED
:1087300009195346CB1A181C291C9846FFF742F911
:10874000071C0198291C784382464046FFF77EF9B2
:1087500036040B04360C33439A4509D91B197A1E8B
:108760009C4200D924E19A4500D821E1023F1B191F
:108770005E4632041743380CBB46009E009F5146AC
:108780003F0C32045B1A5946BA46120C0F043F0CD8
:10879000904651467A434F434146414356467043C3
:1087A000CF19160CBE19B14202D980277F02C01919
:1087B000310C12043604120C4018B618834200D251
:1087C000C4E000D1BEE0191A4846861BB145BF413E
:1087D0007F42CF1BA74200D113E1291C381CFFF7B1
:1087E000F1F8019902904143381C8946291CFFF792
:1087F0002DF9330C0904194389450CD9029B091939
:10880000013B8C4200D9FFE0894500D8FCE0029F83
:108810000919023F02974F46CF1B381C291C0597A8
:10882000FFF7D0F8071C0198291C7843814605986A
:10883000FFF70CF936040904360C0E43B14509D98B
:1088400036197B1EB44200D9E0E0B14500D8DDE026
:10885000023F3619029D4946761A290439430B0412
:1088600057460A0C1B0C40464546584355437B432C
:108870007A43EB18070CDB199D4202D980256D0263
:1088800052191D0C00041B04000C52191B189642AF
:1088900035D300D1FCE001231943049E994FF5190B
:1088A000002D00DCA1E0480709D00F230B40042B6A
:1088B00005D00B1D8B42894149428B44191C5A46F5
:1088C000D20107D5904B5C46049E80271C40FF00D8
:1088D000A346F5198D4B9D427ADD039C012222406F
:1088E00000248B4DA146C1E680242403474627423D
:1088F0004CD13C432403240B009A854DB6E636192F
:10890000481EB4425ED9011C9642C4D1009E9E42CC
:10891000C1D1C2E7031C283B311C99408B46002182
:1089200088E6301C01F0C2F8203072E6283B211C9A
:10893000994000228846914651E6201C01F0B6F885
:1089400020303BE60021B14500D33DE7009F5A4669
:10895000B944B945BF417F423F19FB18013A9C42D7
:108960001ED2984200D97EE000D1B5E0191A934694
:108970002AE7894500D8ADE648464646424677088C
:10898000D3074608C0071E438146AAE65846204240
:1089900012D1044324032A1C240B89465C4D65E64E
:1089A000A342E3D1009F4F45DBD9211A93460BE741
:1089B000171CDDE69B46BCE63C432403240B009ACF
:1089C000534D53E6B24259D800D18AE0011C62E708
:1089D0005F46C9087B07039E0B437C026D0501229D
:1089E0009946240B6D0D324040E64A4B049FDB1B39
:1089F000382B10DD039C0122224000240025A146D3
:108A000034E60121494248E7029304E71F1C21E7AD
:108A1000019C039441E71F2B40DC3F48049F0C1C42
:108A20003A1858469140DC40904020430A1C511EA1
:108A30008A41011C11435A46DA40131C480709D0E9
:108A40000F220A40042A05D00A1D8A428941494260
:108A50005B18111C1A0234D5039C01222240002409
:108A60000125A14602E6009F02214942B9448B44F8
:108A7000B945894149420919CB18A4E6009D881ED1
:108A80006900A942AD416D422C19361900913AE7AF
:108A9000002B00D033E70024009437E71F4A049CE2
:108AA0005D46121BD5402A1C202B1FD01C4E5F4652
:108AB000A3199F403B1C19434B1E994111430023AE
:108AC000BCE75A07C9080A43039F91465B0201228B
:108AD0001C0B3A400025C9E54E45C4D893460021F9
:108AE00072E6009F9F42C9D3011C0FE70023E2E713
:108AF000802424035F463C432403240B019A8946C7
:108B0000034DB3E5FF030000FFFFFFFEFE0700007B
:108B1000FF07000002FCFFFF1E040000E2FBFFFF56
:108B20003E040000F0B55F4656464D464446F0B45C
:108B30000D1C041C8046E80F814618030F03000B30
:108B40003F0B83B084461B48009749005E00DF0F4F
:108B5000490D9246760DBB4681420CD0154886429F
:108B600010D00120B14215D003B03CBC90469946CC
:108B7000A246AB46F0BD009F01202743F4D10D482B
:108B80008642EED1604602430120002AECD101204A
:108B9000B142E9D1009B6345E6D1D045E4D1D94546
:108BA00006D00029E0D11C43201C441EA041DBE775
:108BB0000020D9E7FF070000F0B55F4656464D4656
:108BC0004446F0B4CD0FDE0FAC461D032D0BB1466D
:108BD000374E0F034C00AB465D0080463F0B640DE3
:108BE00092466D0DB44232D0314EB54235D0002C94
:108BF0000ED1384341424141081C002D0BD00029C1
:108C000019D1CC452DD0654668420123184318E0A0
:108C1000002DF6D1281C59460A43534253410028DF
:108C200006D1002BEDD0634658420123184308E0DB
:108C30000020002B05D14A465042504140420123BA
:108C400018433CBC90469946A246AB46F0BD3E1C3C
:108C50000643C9D002204042F3E75E461643C6D021
:108C6000F8E7AC4207DC0BDA614648424841404233
:108C700001231843E5E76646704201231843E0E705
:108C80005F450AD80ED000205F45DAD265466842BB
:108C90006841404201231843D3E762465042012312
:108CA0001843CEE7D045F8D80020D045EED3C8E72A
:108CB000FF070000F0B556464D4644465F46F0B407
:108CC0000D1C83B0041C0190E80F814618030F03AC
:108CD000000B3F0B84463548009749005E00DF0FCC
:108CE000490D9246760DB846814234D02F488642CF
:108CF00036D0002918D0002E1FD1341C67463A43C5
:108D000053425341002C1FD00020002B05D1424676
:108D10005042504140420123184303B03CBC9046AE
:108D20009946A246AB46F0BD0098044360426041BC
:108D3000041C002EE2D00028E9D1C14515D04F46D1
:108D4000784201231843E8E7002BF6D04B465842FF
:108D500001231843E1E7009F02202743DDD1C5E747
:108D6000674602201743D8D1C3E7B14204DD4A4623
:108D7000504201231843D0E7B14207DB0098604519
:108D8000E4D80AD0009F00206745C6D24F467842FB
:108D90007841404201231843BFE7019A5245D5D894
:108DA000019A00205245F1D3B7E7C046FF07000003
:108DB000F0B5564644465F464D46F0B41F1C0B03C3
:108DC0001B0B9A464B0087B0041C80465B0DC80FF6
:108DD000161C02938146002B68D0694B0299994278
:108DE00032D08022534652031A43D200630F1A43F3
:108DF0009246644AE00089188046029100240025CA
:108E00003B031B0B9B467800FB0F321C400D03936A
:108E100000D175E05A4B984269D0802259465203DE
:108E20000A43730FD2001A43564B9346C018F20000
:108E3000002303994E4671401C430F2C00D9A9E032
:108E4000514EA4003459A74653461C4300D087E036
:108E50000025AA46A84608240225D1E74946022D46
:108E60006CD0032D00D117E2012D00D058E10D4048
:108E7000EDB20024A9460023A046002000212503CE
:108E80000A0D1C052D0B1205404B2A4313402343AA
:108E90005B004C465B08E207191C4046114307B0D3
:108EA0003CBC90469946A246AB46F0BD5346234390
:108EB00050D05346002B00D184E1504600F0F6FD1F
:108EC000031E272B00DD76E128210D1A211C083B0B
:108ED0005246E9409A400D1C1543221C9A40AA466E
:108EE00090462B4B00241B1A0293002588E75B4613
:108EF0001E430323002E9CD1B3460022022398E791
:108F00005B46334321D05846002800D14EE100F0A3
:108F1000CDFD272800DD42E128210F1A021C311C5B
:108F2000083A5B46F94093400F1C1F43331C9340A3
:108F3000BB461A1C164B181A00237AE701230B4074
:108F400000249946A0460E4B97E70027BB46002217
:108F500001236EE7002104248A46884601254FE755
:108F60000C2403254CE700258024A9462403A846A9
:108F7000034B82E7DA46904603991D1C6FE7C04613
:108F8000FF07000001FCFFFF3CAA0000FFFF0F806D
:108F90000DFCFFFF029F160C381804904046070C8A
:108FA0000004000C1204120C031C5343041C3D1C4F
:108FB0007443554398463B1C73436419A446444686
:108FC0000293230C63449D4204D9029D80246402D1
:108FD0002D1902951D0C039545462C041B04240CE9
:108FE0001C1905945C46230C051C58432404240CCE
:108FF0008446381C604365435F438146CC44280C5B
:109000006044BB46814502D980277F02BB442D04C2
:10901000070C2D0C000440195546BC462F04E344B0
:109020008446280C3D0C2F1C5743B8462F1C774311
:109030004243B94647463F0C9144BA46D144464361
:109040004A4502D980225202B6184F463A0CB61849
:109050003A0447463F043F0CB8462F1C67435D4324
:109060004443584365190190380C2D184244B846C2
:10907000AC4204D9019880235B02C0180190039C84
:10908000029F201C6044C0196045A44147466442C9
:10909000A4462B043C049946240C4C44A046D844D6
:1090A0008018C246E244904292415746524291464D
:1090B000F219E245BF417F424B46BC46D845BF410D
:1090C000D4187F4263461F432D0C7F19B242924150
:1090D0004C45AD4152426D421543019E7D19AB197D
:1090E000E20D5B02059F134342023A439A46531E28
:1090F0009A41C30D101C1843640220438046504619
:10910000C0010DD5454601225646049C6B082A40F5
:109110001A43F30701341A43760804949046B24682
:10912000049E634FF319002B61DD404640070BD0CE
:109130000F2244462240042A06D0424604324245C9
:1091400080414042824490465546ED0107D5594B37
:109150005646049F80201E40C000B2463B18564A27
:10916000934200DDEAE644465546E20868071043AC
:1091700001226C025B050A408046240B5B0D914680
:109180007BE6DA4690461D1C69E680242403574698
:1091900027421CD13C432403240B484B6DE6031C9F
:1091A000283B311C99408B460022C3E6301C00F05E
:1091B0007DFC2030ADE6283B211C994000228A46E8
:1091C00090468EE6201C00F071FC203078E6584670
:1091D000204207D1044303992403240B8946904677
:1091E000364B4AE63C432403240B344B45E6344BD0
:1091F000049E9B1B382B06DD01230B40002499465F
:10920000A046002339E61F2B25DC049C2D4D464645
:109210006019524644468640DC4082405746301C26
:109220002243DF40441EA04102433B1C540709D0A7
:109230000F201040042805D0101D90429241524248
:109240009B18021C1D021AD501230B4000249946CD
:10925000A046012311E61C48049C5546001BC5404E
:10926000281C202B16D0194E5746A21997403A1C9D
:1092700043461A43531E9A4102430023D6E7580738
:109280005B02D2081C0B01230B4010439946804619
:109290000023F2E50022EBE780242403504601235B
:1092A000044319402403240B8946044BE5E5C046DA
:1092B000FF030000FFFFFFFEFE070000FF070000A6
:1092C00002FCFFFF1E040000E2FBFFFF3E04000063
:1092D000F8B55F46564644464D46F0B40C034D0083
:1092E000CF0F610A440F2143C4001803DE0F8046EC
:1092F000B44646465800760A530F3343D600C94A4F
:109300006D0DBA46400DB346904200D1EBE0624687
:10931000012672409446674500D1A1E02F1A002F24
:1093200000DC08E100283BD15846184300D0E8E0B3
:10933000600709D00F232340042B05D0231DA3422F
:10934000A441644209191C1C0A0200D479E0B54BFF
:109350006A1C9A4200D109E1B34BE408194048075E
:10936000044349025205012750460B0B520D07409A
:10937000002000211B03201C1C0B0B0D1B05AB4DFB
:109380002343520552081D4015436D006D08FF0729
:10939000291C39433CBC90469946A246AB46F8BDD1
:1093A000A0488542C4D0802000040343382F00DD4C
:1093B000F0E01F2F00DD24E12020C01B1A1C5E46B8
:1093C0008240FE40324394465A468240101C421E60
:1093D0009041FB40624602431F1CA21A9442A441E2
:1093E0006442C91B091B141C0A02A1D549024F0A79
:1093F000002F00D1C9E0381C00F058FB021C083ACD
:109400001F2A00DDBCE02821231C091A9740CB400D
:109410001F439440954200DDAEE0551B691C1F2997
:1094200000DDDDE01F22551B3B1C221CAB40CA4067
:10943000AC40651EAC411343CF401C43391C002592
:1094400076E74807E4086A0501275646C908520D21
:1094500037400443734B9D4249D009030B0B87E708
:109460002A1A9446002A00DC9BE0002855D06D485B
:10947000854200D15CE78020000403436046382821
:1094800000DD09E11F2800DD50E162462020801A3E
:109490001E1C8640B1465E46D6404A4632435E4672
:1094A00086409046301C421E904142460243604630
:1094B000C3401219A242A441644259180919141C4C
:1094C000080200D434E7574B01359D4200D142E1F8
:1094D000554B60081940012323401C1C0443CB0753
:1094E0001C43490824E71E4300D014E70FE70B1C78
:1094F000234300D1CFE180231B030B431B031B0B32
:1095000036E7013F002F66D15E46A21B9442A4417C
:109510006442C91A091B141C66E75846184300D157
:1095200006E701267642B4446046002800D0CAE02F
:109530005E463219BEE7002F7AD1681C4005400D07
:10954000012800DCE3E05A46A21A9442BF41C81A3F
:109550007F42C71B3E0200D492E05846041BA3453D
:109560009241591A52428F1AE24641E75346012767
:109570001F4000240023FBE62B49AD1A3940D7E6F3
:10958000271C28388740002444E7201C00F08EFA6E
:10959000203033E75A461A43531E9A41D2B200276D
:1095A0001BE7002A00D0E1E0681C4605760D012E7D
:1095B00000DC91E01B4DA84200D1F7E05E46321975
:1095C000A242A441644259180919CC075208144315
:1095D0004908051CACE61348854200D0E6E6A7E63C
:1095E0002B1C1F3B3E1CDE40331C202970D03F2229
:1095F000551BAF403C43601E84411C4300210025A5
:1096000096E6381C20381E1CC640301C202F61D026
:109610004022D71BBB405A461A43531E9A4102436D
:109620000027DAE6FF070000FFFF7FFFFFFF0F8044
:10963000002D38D0B94DA84200D192E080252D04EC
:109640007F422943382F00DDAAE01F2F00DD2CE1E7
:109650002025ED1B0E1CAE40B046261CFE404246A7
:10966000AC401643651EAC413443F9405A46141BC6
:10967000A34592415B1A5242991A051CE246B3E691
:10968000131C3B43141C002B00D0B1E60027002222
:10969000002500210024DDE65A461A43531E9A4154
:1096A000D2B2002305E70D1C25435AD0FF43002FFB
:1096B00053D15A46141BA3459241591A5242891A52
:1096C000051CE24690E69548854200D0D6E62FE696
:1096D00000278FE700239EE7081C2043002D00D0C1
:1096E000C3E0002800D1F6E05846184300D11FE639
:1096F00058460219A242A441644259180919141C7F
:109700000A0200D414E6864B0125194010E6081C15
:109710002043002D3AD1002800D089E05946194352
:1097200000D1BFE0191C5C46E24601E660462038E5
:109730001A1CC2406646101C202E00D1B0E0402208
:10974000921B93405A461A43531E9A4102430023E8
:10975000AFE6724D00272A1C9BE7704DA84200D04F
:1097600070E7191C5C46051CE246E1E5002D20D19E
:109770000D1C254375D0D543002D6FD15C445C454D
:109780009241591852428918051C99E6002835D192
:1097900059461943DDD0191C5C46E2465F4DC7E5CA
:1097A0000C43611E8C41E4B200215FE7051C021CE2
:1097B0006FE75A4DA84254D05542802216043143D7
:1097C000382D00DD81E01F2D00DD91E02022561BA9
:1097D0000A1CB446B240261CEE4032439046624614
:1097E0009440661EB44142461443E9405C445C45E3
:1097F0009241CB1852429918051C61E6584618430D
:109800004CD04807E40804438020C9080003014203
:1098100008D0DD08054205D15946CA085C07144343
:10982000291CE246630FC9001943E4003B4D7FE564
:109830005846184300D17BE55E46A71BBC429241C7
:10984000C81A5242801A06024CD55846041BA3453A
:109850009241591A5242891AE24669E52F4A9042CA
:10986000AED1191C5C46051C62E5002836D058466E
:10987000184313D080254807E408C9082D03044382
:109880002942CFD0D8082842CCD15D46EA085C07EF
:109890001443011CC6E70023002469E51F4D47E57A
:1098A00000234FE700270022F3E63D1C203D0E1C5D
:1098B000EE40351C202F2DD04026F71BB9400C431D
:1098C000611E8C412C430021D0E60C43611E8C416B
:1098D000E4B200218AE7191C5C4629E5191C5C46A4
:1098E0000E4D25E5031C3B43DCD0011C3C1C1FE551
:1098F0002026764276190A1CF2409046202D0BD085
:109900004026751BA9400C43611E8C4145462C43E3
:1099100000216BE70021D2E70021F4E7FF070000F8
:10992000FFFF7FFF70B50B1C124C09030E0B590093
:10993000021C490DDD0F0020A14211DD0E488142BD
:109940000FDC8020400306430C48401A1F280BDD23
:109950000B4A521AD640321C5042002D00D1101C26
:1099600070BD084BE818FBE7074BC240C9188E4092
:109970003243F1E7FE0300001D0400003304000041
:1099800013040000FFFFFF7FEDFBFFFFF8B5041E8F
:1099900031D0C70F00D04442201C00F087F8184D8A
:1099A0002D1A0A2819DD0B38844024036D05240B79
:1099B0006D0D3A1C0026002000210B0D2403240B02
:1099C0001B0523430F4C2D051C402C4364006408E9
:1099D000D307211C301C1943F8BD061C1536231C67
:1099E000B3401E1C0B23181AC44024036D05240B1E
:1099F0006D0D3A1CDFE70022002500240026DAE77F
:109A00001E040000FFFF0F8043001B0E5A1C410282
:109A1000D2B270B54C0AC50F012A17DDE0229200C0
:109A20006407090B9818002200231E0D221C340520
:109A30000C431B49400540082140014349004908A7
:109A4000ED070B1C2B43101C191C70BD002B15D1EE
:109A5000002C1CD0201C00F029F80A281ADC0B214D
:109A6000091A231CCB40191C031C15339C400D4BB9
:109A70000903181A4005090B400DD4E7002C03D048
:109A80006407090B0848CEE707480021CBE7002010
:109A90000021C8E7011C0B398C40211C0024E6E79B
:109AA000FFFF0F8089030000FF0700001C21012336
:109AB0001B04984201D3000C10391B0A984201D3B1
:109AC000000A08391B09984201D30009043902A28F
:109AD000105C40187047C0460403020201010101F6
:109AE000000000000000000010B5F9F77BF9F9F75D
:109AF00051F9F8F715FFF8F729FFF8F755FFF8F7D0
:109B00009FFFF8F7B1FFF9F723FB164C1649201C0D
:109B1000F9F7DEFCA078A188A289F9F767F9134C60
:109B20002378002B16D0F9F705F9F9F7ADFB104BA8
:109B300001221A70FBF748FCF9F764FEF9F734F8D4
:109B4000F8F7CAFFFDF724FF0120FDF7DFFDFBF763
:109B500089FBF7E7F9F7AAF82378002BE3D1F9F7A7
:109B6000A5F8E0E7F4F0FF1FB8F0FF1FB5F0FF1F06
:109B7000F0F0FF1FF8B54E001B4F760DF319132BB5
:109B800011DC002B05DACB0FDD07002414605560D3
:109B900029E0164E1E41331C0B40034313D00F1C0B
:109BA000B743002619E0332B05DDCB0F1060516061
:109BB000D907002017E00E4F0123F6195B42F3404E
:109BC0009C46034005D110605160CA0FD107181C94
:109BD00009E0061C63460F1C9E43166057603B1C41
:109BE000321CFFF775FBF8BD01FCFFFFFFFF0F0004
:109BF000EDFBFFFF00000000F0B556464D46444621
:109C00005F46F0B4504A4F007F0D83B0BE18041C6D
:109C10000D1C89468A4680460197132E2FDC002EA4
:109C200068DB4A4F021C37413B1C0B4003439C46F8
:109C3000BB4667460B1C002F18D0404B3E4AFEF730
:109C400031F93F4A3F4BFDF797FF00280CD0002D1C
:109C500004DD80235B0333415E19B24653465F4601
:109C6000BB430022994690464B464246101C191CA5
:109C700003B03CBC90469946A246AB46F0BD332E9D
:109C80000BDD0B1C8021021CC9008E42EED1291C69
:109C9000FEF708F9021C0B1CE8E7019F2C4ABB18D1
:109CA00001225242DA4093465F46021C0B1C0742D7
:109CB000DCD0224B204AFEF7F5F8214A214BFDF774
:109CC0005BFF0028D0D0002D0CDD142E2ED0214BB0
:109CD000019A9F1A0123BB401F19BC421ED96B1C5D
:109CE0009A46B84647465A469743B846D1464B46E9
:109CF0004246BBE7114B104AFEF7D4F8104A114B0D
:109D0000FDF73AFF0028AFD0002D09DB00272C43D8
:109D1000B846B946A8D0104A9146A5E7B846E1E74B
:109D20000023984680231B0699469DE76B1C9A46A4
:109D3000D8E7C046C046C0469C7500883CE4377EE4
:109D4000000000000000000001FCFFFFFFFF0F000B
:109D5000EDFBFFFF330400000000F03FC046C046AB
:109D6000F0B556464D4644465F46F0B4524A4F0061
:109D70007F0D83B0BE18041C0D1C89468A468046A0
:109D80000197132E2ADC002E56DB4C4F021C374164
:109D90003B1C0B4003439C46BB4667460B1C002FF5
:109DA00013D0424B404AFEF77DF8414A414BFDF744
:109DB000E3FE002807D0002D4EDB53465F46BB4331
:109DC0000022994690464B464246101C191C03B08F
:109DD0003CBC90469946A246AB46F0BD332E0BDD07
:109DE0000B1C8021021CC9008E42EED1291CFEF7FB
:109DF00059F8021C0B1CE8E7019F314ABB180122ED
:109E00005242DA4093465F46021C0B1C0742DCD0EC
:109E1000264B254AFEF746F8254A264BFDF7ACFEB1
:109E20000028D0D0002D1DDB42465B469A43904669
:109E3000D1464B464246C8E71C4B1B4AFEF732F858
:109E40001B4A1C4BFDF798FE0028BCD0002D17DBE9
:109E50000027B846B946B6E780235B0333415E1955
:109E6000B246AAE7142E19D0164B019A9F1A012365
:109E7000BB401B199C420FD96F1CBA469846D3E7CA
:109E80006B005B081C4302D10027B8469BE70E4FCE
:109E900000239846B94696E79846C5E76B1C9A4654
:109EA000C2E7C046C046C0469C7500883CE4377E89
:109EB000000000000000000001FCFFFFFFFF0F009A
:109EC000EDFBFFFF330400000000F0BFC046C046BA
:109ED0003A2700003A270000F4260000A6260000DA
:109EE000A6260000622700009300222000009400B4
:109EF00000000001809698000000010001000300AE
:109F0000040004000000010002000300040004003B
:109F10000100010002000100010001000000010039
:109F20000100030004000400000001000100030020
:109F300004000500040004000400040004000500FF
:109F4000809F0000789F0000709F0000689F0000C5
:109F5000609F0000589F0000A01000809400000047
:109F6000A000008094000000200000809400000009
:109F70004410008000000000440000800000000049
:109F80000400008000000000142C00001E2C0000C3
:109F9000282C0000322C0000002C00000A2C0000AD
:109FA0000B0000002A2E00002A2E0000862E000042
:109FB0008E2E0000962E00009E2E00002A2E0000FD
:109FC0007E2E0000A62E0000030101020702000001
:109FD0000000000000000000020201020202000076
:109FE0000000000000000000030301020202020260
:109FF000020202020203000000000002030100004E
:10A000000303020101000000000000000000000046
:10A010000000000000000000000000000000000040
:10A020000000000000000000020202020202020220
:10A03000020201010302020102010201000000000C
:10A040000000000000000000F6420000564300003F
:10A050007C43000096430000AC4300003A440000FB
:10A06000F642000052440000F6420000F6420000B2
:10A07000C6430000E0430000C842000082440000E4
:10A0800042430000A8460000F642000028450000B8
:10A090004A450000C0440000DC440000F8440000D1
:10A0A0000A45000066450000A0450000FA45000092
:10A0B0003E4600004A460000F6420000A04600006E
:10A0C00042430000A8460000784900008A49000089
:10A0D0009C490000AE490000C4490000D849000076
:10A0E000EA490000FC490000524900006A490000AA
:10A0F000644A0000724A0000804A00008E4A000054
:10A10000A04A0000B04A0000BE4A0000CC4A00004D
:10A11000DA4A00003E4A0000564A0000344B000074
:10A12000404B00004C4B0000584B0000284B0000F7
:10A130001C4B0000484D0000344D00003E4D000017
:10A14000524D00005C4D0000664D0000724D000055
:10A150007C4D0000864D0000904D00009A4D00009F
:10A160002A4D0000144D00002C550000F460000042
:10A17000385E000078600000D05B0000C060000026
:10A18000E45C00004E5F0000745A0000186000009C
:10A190007A5D0000F45F00003A5B00009E60000002
:10A1A000725C0000CC5E0000005A000054600000A9
:10A1B000F85D0000A45F0000785B000034600000E0
:10A1C000AC5C00000E5F00003C5A00003A5D0000ED
:10A1D000005B0000E65A0000CC5A00007A5E0000E6
:10A1E000126100001C5C000012610000126100009E
:10A1F0001261000012610000126100001261000093
:10A200001261000012610000665900001261000036
:10A210001261000012610000126100001261000072
:10A220001261000012610000126100001261000062
:10A230001261000012610000126100001261000052
:10A240001261000012610000126100001261000042
:10A250001261000012610000126100001261000032
:10A260001261000012610000126100001261000022
:10A270001261000012610000126100001261000012
:10A280001261000012610000126100001261000002
:10A2900012610000126100001261000012610000F2
:10A2A00012610000126100001261000012610000E2
:10A2B00012610000126100001261000012610000D2
:10A2C00012610000126100001261000012610000C2
:10A2D00012610000126100001261000012610000B2
:10A2E00012610000126100001261000012610000A2
:10A2F0001261000012610000126100001261000092
:10A300001261000012610000126100001261000081
:10A310001261000012610000126100001261000071
:10A320001261000012610000126100001261000061
:10A330001261000012610000126100001261000051
:10A340001261000012610000126100001261000041
:10A350001261000012610000126100001261000031
:10A36000126100004E5900001261000012610000ED
:10A370001261000012610000126100001261000011
:10A380001261000012610000126100001261000001
:10A390001261000012610000CA5F0000126100003B
:10A3A00012610000126100001261000012610000E1
:10A3B00012610000126100001261000012610000D1
:10A3C0001E5E0000345F00009A5B0000B25E000079
:10A3D000CA5C0000965E00005C5A00005E5D0000F2
:10A3E000445C00005C5C000012610000126100002F
:10A3F000205B0000E6590000CC590000A459000081
:10A400007C590000BC5D00009E5D0000DA5D00002C
:10A410005E5B00007A5F0000925C0000F05E00006E
:10A42000225A000012610000126100005C5E000010
:10A43000126100000E5D0000AE5A0000925A00004A
:10A440002C5900001261000012590000025C00004B
:10A45000DA58000072580000E05700005858000019
:10A46000565700003C57000006570000D856000021
:10A47000A0560000A2580000FA5700008C580000B7
:10A4800012610000126100001261000020570000FC
:10A49000945700007A570000C65700001261000070
:10A4A00082560000D6550000BE5500006A560000D6
:10A4B0008E55000012610000385600001261000045
:10A4C0000A560000126100001261000012610000D3
:10A4D00012610000126100001261000012610000B0
:10A4E00012610000126100001261000012610000A0
:10A4F0001261000012610000126100001261000090
:10A50000126100001261000012610000126100007F
:10A51000126100001261000012610000126100006F
:10A52000126100001261000012610000126100005F
:10A53000126100001261000012610000126100004F
:10A54000126100001261000012610000126100003F
:10A55000126100001261000012610000126100002F
:10A56000625500004C550000867100009A71000091
:10A57000B2710000CC710000E871000000720000B0
:10A580001472000026720000327200003E72000059
:10A59000447200007A720000AE720000B6720000D1
:10A5A000B6720000B6720000B6720000B67200000B
:10A5B000B6720000B67200007E710000EE760000F8
:10A5C000E8760000E2760000DC760000D676000037
:10A5D000D0760000D0760000D0760000D076000063
:10A5E000CA760000CA760000EE760000EE76000023
:10A5F000C4760000EE760000BE760000EE76000025
:10A60000EE760000EE760000B8760000B27600002C
:10A61000AC760000A6760000A07600009A760000D6
:10A62000EE760000EE760000947600008E76000054
:10A63000EE76000088760000827600007C760000CE
:10A6400076760000707600006A760000647600007E
:10A65000EE760000EE7600005E760000EE760000FA
:10A66000EE760000EE760000EE760000EE7600005A
:10A67000EE760000EE760000EE760000EE7600004A
:10A68000EE760000EE760000EE760000EE7600003A
:10A69000EE760000EE760000EE760000EE7600002A
:10A6A000EE760000EE760000EE760000EE7600001A
:10A6B000EE760000EE760000EE76000058760000A0
:10A6C000EE760000EE760000EE760000EE760000FA
:10A6D000E0750000EE760000E0750000EE76000008
:10A6E000EE760000EE760000EE760000EE760000DA
:10A6F000EE760000EE760000EE760000EE760000CA
:10A70000EE760000EE760000EE760000EE760000B9
:10A71000EE760000EE760000EE760000EE760000A9
:10A72000EE760000EE760000EE760000EE76000099
:10A73000EE760000EE760000EE760000EE76000089
:10A74000EE760000EE760000EE760000EE76000079
:10A75000EE760000EE760000EE760000EE76000069
:10A76000EE760000EE760000EE760000EE76000059
:10A77000EE760000EE760000EE760000EE76000049
:10A78000EE760000EE760000EE760000EE76000039
:10A79000EE760000EE760000EE760000EE76000029
:10A7A000EE760000EE760000EE760000EE76000019
:10A7B000EE760000EE760000EE76000052760000A5
:10A7C0004C760000467600004076000032760000AD
:10A7D000287600001C760000167600001076000037
:10A7E0000A760000EE760000EE76000004760000A7
:10A7F000FE750000EE760000EE760000EE760000BA
:10A80000EE760000F4750000EE760000E8750000BA
:10A81000EE760000EE760000EE760000EE760000A8
:10A82000EE760000EE760000EE760000EE76000098
:10A83000EE760000EE760000EE760000EE76000088
:10A84000EE760000EE760000EE760000EE76000078
:10A85000EE760000EE760000EE760000EE76000068
:10A86000EE760000EE760000EE760000EE76000058
:10A87000EE760000EE760000EE760000EE76000048
:10A88000EE760000EE760000EE760000EE76000038
:10A89000EE760000EE760000EE760000EE76000028
:10A8A000EE760000EE760000EE760000EE76000018
:10A8B000EE760000EE760000EE760000EE76000008
:10A8C000EE760000EE760000EE760000EE760000F8
:10A8D000EE760000EE760000EE760000EE760000E8
:10A8E000EE760000EE760000EE760000EE760000D8
:10A8F000EE760000EE760000EE760000EE760000C8
:10A90000EE760000EE760000EE760000EE760000B7
:10A91000EE760000EE760000EE760000EE760000A7
:10A92000EE760000EE760000EE760000EE76000097
:10A93000EE760000EE760000EE760000EE76000087
:10A94000EE760000EE760000EE760000EE76000077
:10A95000EE760000EE760000EE760000EE76000067
:10A96000EE760000EE760000EE760000EE76000057
:10A97000EE760000EE760000EE760000EE76000047
:10A98000EE760000E2750000EE760000EE76000044
:10A99000EE760000EE760000EE760000EE76000027
:10A9A000EE760000EE760000EE760000EE76000017
:10A9B000EE760000EE760000D4750000EC7C00001E
:10A9C0009E7C0000CC7C0000267C0000CC7C00003B
:10A9D000C27C0000CC7C0000267C00009E7C000035
:10A9E0009E7C0000C27C0000267C00001E7C0000D3
:10A9F0001E7C00001E7C0000D27C0000C48600008B
:10AA000060860000A88600008E850000A8860000F1
:10AA10009C860000A88600008E85000060860000ED
:10AA2000608600009C8600008E8500008485000002
:10AA30008485000084850000E8880000948F000071
:10AA40008291000082910000748F00005E8E0000F1
:10AA50005E8E0000668F0000748F00005E8E000026
:10AA6000668F00005E8E0000748F00005C8E000018
:10AA70005C8E00005C8E00008A910000313237301D
:10AA80005631303000000000F8B5C046F8BC08BCB4
:10AA90009E467047F8B5C046F8BC08BC9E46704755
:04AAA0003924000055
:04AAA4001124000079
:08AAA800010000007CAA00007F
:10AAB000A8AA000008F0FF1F080000000000000026
:08AAC00000000000000000008E
:020000041FFFDC
:04F00000000000000C
:040000030000289938
:00000001FF
